:100000000C94A4040C94C1040C94C1040C94C10479
:100010000C94B8140C94C1040C94C1040C94C10445
:100020000C94C1040C94F6050C94C1040C948A063B
:100030000C94C1040C94C1040C94C1040C94C1042C
:100040000C94C1040C94C1040C94C1040C94C1041C
:100050000C94C1040C94C1040C94C1040C94C1040C
:100060000C94C1040C94C104E10B1F0C320C5F1101
:100070005F115F115F115F115F115F115F115F1100
:100080005F115F115F115F115F115F115F115F11F0
:100090005F115F115F115F115F115F11370C5F110D
:1000A0005F0C730C8E0CB60CE40CF50C090D330DC3
:1000B0005F0D5F0D670E670E670E670EDE0BA40EF9
:1000C000680D7F0D870F910F121012101210121071
:1000D00012105F115F115F115F115F115F115F11EE
:1000E0005F11A60FFC0F12106364696E6F70737559
:1000F00078585B003C656D7074793E20202020208C
:10010000006572726F723A20777269746520616659
:1001100074657220666F726D61740053494F2D458E
:1001200072726F723A2025690053494F3A434D4429
:100130002054696D656F75740053796E6320576143
:1001400069742E2E2E2020200053746F7070656409
:100150002E2E2E202020003E4E65773C2020202091
:10016000202020004572726F7220696E69742046EB
:1001700041543A20257500252E30386C7820252EE4
:1001800030386C78004572726F7220696E69742025
:1001900053443A202575005344524956452E415444
:1001A00052206E6F7420666F756E6400252E327853
:1001B00020252E327820252E327820252E327820C8
:1001C0002563202575006572726F723A206372652F
:1001D000617465206E65772066696C65000F111388
:1001E00015181A1C1E212325325344726976653175
:1001F00033203230323231323034206279204B4277
:1002000072006279204B42722056312E33005344E3
:10021000726976652D4D41580053444D58252E3452
:10022000750053444D58256875004154520054469A
:10023000542D49443A20252E30347800546170659D
:100240002D456D750058313A2025692C2058323AD9
:100250002025692C2059313A2025692C2059323A21
:100260002025690020202020202020202020202060
:100270000025692066696C65732C207061676520B4
:1002800025692F256920202573202020202020206B
:10029000202020202000C50100000000F0001801EF
:1002A00059CE0000FFFF1E011A2059010F00A500C2
:1002B00050001E0059CE0000FFFF220171205F0197
:1002C0000F00CD0050001E0059CE0000FFFF21019D
:1002D000D32365019000A50050001E0059CE0000F8
:1002E000FFFF2001B8236B019000CD0050001E00DD
:1002F00059CE0000FFFF1F011A2070010F002D00D2
:100300005A001E0059CE00001F052A01F123770173
:100310000F0055005A001E0059CE00001F0529018C
:10032000F1237E010F007D005A001E0059CE00000F
:100330001F052801F12385010F00A50046001E00BE
:1003400059CE00001F052701F1238A010F00CD00BF
:1003500050001E0059CE00001F052601F123900118
:100360000F00F5005A001E0059CE00001F052501A0
:10037000F1239701A4007D003C001E0059CE00002F
:10038000FFFF2401A2276B01A400A5003C001E0072
:1003900059CE0000FFFF23011A209C01A4002D006C
:1003A0003C001E0059CE0000FFFF31019721A00143
:1003B000A40055003C001E0059CE0000FFFF300194
:1003C0008621A501A4007D003C001E0059CE00003E
:1003D000FFFF2F0139206B01A400A5003C001E0087
:1003E00059CE0000FFFF2E011A20A801A400CD0065
:1003F0003C001E0059CE0000FFFF2D01A220AD01E0
:10040000A400F5003C001E0059CE0000FFFF2C01A7
:10041000A021C5010F002D009600F00059CE00006C
:10042000FFFF2B01A726B2010A00C80032001E0000
:1004300059CE000000003A01FF1FB6010A00280053
:10044000DB001E0059CE0000000039017420C601F7
:100450000A005000DB001E0059CE000000003801E9
:100460007420D6010A007800DB001E0059CE00007F
:10047000000037017420E6010A00A000DB001E0026
:1004800059CE0000000036017420F6015000C8006B
:1004900050001E0059CE0000000035010920FC016B
:1004A000B300C80032001E0059CE0000E00734013E
:1004B000712000020A00F00032001E0058540000B3
:1004C000DFFF330171200402B300F00032001E0090
:1004D00059CE00001F0032016320C5010A00180137
:1004E000E5003F01000000000000220239264154CF
:1004F00052415458434153434F4D42494E4558454C
:10050000584558584644544150494D47424153522A
:10051000454144590000002421E318C318E318049E
:100520002104210000000000000000000000000085
:1005300000000000000421821041084108410861C8
:100540000861084569456982108210A210A210C393
:1005500018042100008210410820002000200041E2
:100560000841084569456941084108610841086139
:1005700008821000008210200020002000200020AF
:100580000041084569456941084108410841084161
:10059000086108A2108210200020002000200041E5
:1005A0000861086108610861086108610861084123
:1005B000086108A210A21041082000200041086133
:1005C000088210FFFFFFFF0000A210A2108210613E
:1005D000088210A210C318610841084108821082E5
:1005E00010FFFF1F001F00FFFF0000E318A2108292
:1005F000108210C318E3188210610861088210FF8E
:10060000FF1F001F001F001F00FFFFC318A2108262
:10061000108210C318E318821082108210A210FFFB
:10062000FF1F001F001F001F00FFFFC318A2106163
:10063000088210C318C318821061088210A210E348
:1006400018FFFF1F001F00FFFF0000A210821061B3
:10065000086108A2108210610841088210C31804C2
:10066000212421FFFFFFFF0000C318A210821041C8
:1006700008610882101F000000200041088210C39A
:1006800018E318E318E318C318C318A2106108612F
:10069000086108610800000000200041086108A20C
:1006A00010C318C318A210A210A210821061084132
:1006B00008610882106108000020002000610882A3
:1006C00010A210A2108210821082106108610861CD
:1006D000088210A210C3186108410841086108820D
:1006E00010A210A21082108210821082108210823A
:1006F00010C318000000000000000000000000000F
:1007000000000000000000000000000000000000E9
:100710000000000000001705183419011FD4283C00
:10072000000000000000005F000000070007001448
:100730007F147F14242A7F2A122313086462364907
:100740005522500005030000001C224100004122F8
:100750001C0014083E081408083E08080050300029
:100760000008080808080060600000201008040263
:100770003E5149453E00427F400042615149462179
:1007800041454B311814127F1027454545393C4AE5
:100790004949300171090503364949493606494935
:1007A000291E00363600000056360000081422418B
:1007B00000141414141400412214080201510906F3
:1007C000324979413E7E1111117E7F494949363EB9
:1007D000414141227F4141221C7F494949417F09D2
:1007E0000909013E4149497A7F0808087F00417F95
:1007F00041002040413F017F081422417F4040409A
:10080000407F020C027F7F0408107F3E4141413E41
:100810007F090909063E4151215E7F091929464693
:100820004949493101017F01013F4040403F1F20BC
:1008300040201F3F4038403F63140814630708708E
:1008400008076151494543007F41410002040810F7
:10085000200041417F00040201020440404040402A
:10086000000102040020545454787F48444438382E
:1008700044444420384444487F3854545418087E33
:1008800009010218A4A4A47C7F0804047800447D14
:1008900040004080887A007F1028440000417F405B
:1008A000007C041804787C080404783844444438F4
:1008B000FC2424241818242418FC7C080404084868
:1008C00054545420043F4440203C4040207C1C2091
:1008D00040201C3C4030403C44281028441CA0A030
:1008E000A07C4464544C44000836410000007F0062
:1008F0000000413608001008081008784641467884
:10090000FFFFFFFFFF426C6F636B202575202020E7
:10091000202000426175643A202575204C656E6781
:1009200074683A202575204761703A20257520208B
:10093000202000456E64202000426C6F636B2025F0
:1009400075202F202575200011241FBECFEFD8E081
:10095000DEBFCDBF12E0A0E0B1E0E4E2FCE702C000
:1009600005900D92A830B107D9F726E0A8E0B2E0D3
:1009700001C01D92A33EB207E1F70E9474110C94CE
:10098000103E0C9400000F931F939091210291113F
:1009900031C0E0914001F09141012281338194E125
:1009A000899F200D311D1124F9017096A591B491F4
:1009B0008C9182FF03C00FE110E002C009E51EEC3C
:1009C000462FF9013296849190E032962491622F5D
:1009D00070E06B5F7F4F0596413029F0423029F47B
:1009E00000E018EF02C000EE17E021E043E050E025
:1009F0000E94002B1F910F910895CF93DF9340E049
:100A000050E090E060E3680F71E3E0914001F09105
:100A100041010280F381E02D9F01240F351FF90170
:100A20007096C591D491F901A591B49128812B7F3D
:100A30002883891302C02460288320E3290F11969C
:100A40002C931197823048F0891303C011967C9340
:100A500004C0913011F411966C939F5F4C5E5F4F10
:100A6000953099F680912102811102C00E941B23CA
:100A7000DF91CF910895A0E1B0E0E1E4F5E00C94BE
:100A800026356B017C018E010F5F1F4F80E1F8015D
:100A900011928A95E9F7C701B601605F7F4F8F4FCA
:100AA0009F4F0E94791E611571058105910569F1BD
:100AB00026E932E03A8329834601570124E0B694BF
:100AC000A794979487942A95D1F79C828B82F1E022
:100AD000CF16F8E0DF06F2E0EF06F10418F020E0B0
:100AE00031E002C020E830E03E832D830E94DE1614
:100AF00080E1F801A4EBB2E001900D928A95E1F754
:100B000080E00E949E1680E005C086EC91E00E9485
:100B1000A92581E06096ECE00C944235E62FF0E0E8
:100B2000EC54FB4F6AE00E947434806380839063CE
:100B300091830895E4EBF4E08C549B4F1192E817F5
:100B4000F907E1F708959091B5059F939091B40549
:100B50009F931F928F93ECEDF5E083811F928F930B
:100B600082811F928F9381811F928F9380811F9228
:100B70008F938CEA91E09F938F9388EC95E09F93FD
:100B80008F930E94E13788EC95E00E947F268DB715
:100B90009EB740960FB6F8949EBF0FBE8DBF0895C6
:100BA00080E090E00E94DA29E0E7F0E08081816057
:100BB0008083E1EBF0E08081876080830895E0E747
:100BC000F0E080818E7F80831092B10080912102BD
:100BD000E0914001F091410195E0899FE00DF11D08
:100BE00011240190F081E02D099508951F920F9234
:100BF0000FB60F921124EF92FF920F931F932F9332
:100C00003F934F935F936F937F938F939F93AF9394
:100C1000BF93CF93DF93EF93FF93809108028F5F91
:100C2000809308028F7309F50E94B337EC010E948C
:100C3000B3378C0180E090E00E94DA29C8016CE2B1
:100C400071E00E949434FC01CE0168E770E00E94DC
:100C500094342EE0E22E22E0F22E00E010E028E0B4
:100C60003CEF42E0BF010E94502CFF91EF91DF91D9
:100C7000CF91BF91AF919F918F917F916F915F9134
:100C80004F913F912F911F910F91FF90EF900F90F7
:100C90000FBE0F901F9018950F931F9380910D0218
:100CA00081111EC0E091BE05F091BF05868981FFCC
:100CB00009C02FE781E397E1215080409040E1F7A0
:100CC00000C000008BE08093810000EE17E021E07F
:100CD00043E050E065E070E085E090E00E94002B8A
:100CE00081E080930D021F910F9108950F931F9340
:100CF0001092810010920D0200E010E021E043E02C
:100D000050E065E070E085E090E00E94002B1F91CC
:100D10000F9108951F920F920FB60F9211242F93E7
:100D20003F934F935F936F937F938F939F93AF9373
:100D3000BF93EF93FF9380910D02882319F08F5F8B
:100D400080930D0280910D02853110F00E9476068D
:100D5000FF91EF91BF91AF919F918F917F916F9193
:100D60005F914F913F912F910F900FBE0F901F9069
:100D70001895A0E0B0E0EFEBF6E00C942B358CE397
:100D800092E09093BF058093BE05809138029091C8
:100D90003902A0913A02B0913B02809340029093B5
:100DA0004102A0934202B0934302E12CF12C60E097
:100DB000C7010E949518882309F45CC004EB14E075
:100DC000C1E6D0E0F801D1908F01CE010E94C83D6C
:100DD000D8124CC02196F4E00F3B1F0799F7E09121
:100DE000BE05F091BF0580819181A281B38180878A
:100DF0009187A287B387148615861686178620E109
:100E000030E040E050E0BA0180E00E949D1AC091BD
:100E1000BE05D091BF0581E08E8B9091B804809182
:100E2000B904892B813011F481E28E8B8A899B89E8
:100E3000AC89BD89BC01CD0160517109810991095D
:100E40001E8915FD05C020E830E040E050E004C0F8
:100E500020E031E040E050E00E94A834213D3240E3
:100E60004105510580F010681E8B0DC0EFEFEE1AA2
:100E7000FE0A9DCFE091BE05F091BF05168A87E975
:100E800091E00E94A925CDB7DEB7E7E00C94473585
:100E9000A7E0B0E0EEE4F7E00C9420358091DD05AA
:100EA000811155C040E064E070E08CED95E00E9457
:100EB0004C1F823031F489E291E00E94A9250C9404
:100EC0007011AFE7BCE01197F1F700C00000359B4F
:100ED000FECF882309F43BC090910F029923B1F013
:100EE0001F928F938BE191E09F938F9384EB94E01B
:100EF0009F938F930E94E13784EB94E00E947F26BA
:100F00000F900F900F900F900F900F908091C2054F
:100F1000883239F081E09091C105911180E0809391
:100F2000C1058091C105882361F0E091C205EB30D5
:100F300018F0E8EEF1E003C0F0E0E352FE4F8491D8
:100F400001C088E690E00E94181F0C947011109167
:100F5000DD058091DC059FEC980F943080F42091A2
:100F6000C005813319F42093B6051AC090E030E033
:100F7000205D3F4F8217930771F481E00FC08137E6
:100F800011F00C94701180EB810F843008F0FAC3DB
:100F900080E38093DC058091DC058F708093B6053B
:100FA0008091B605482F50E0B8E18B9FF0011124E5
:100FB000E45CFD4FF093BF05E093BE059689292FB1
:100FC000297011F40C947011133509F40AC1292FFA
:100FD0002B7F268B123209F4DCC018F4113241F059
:100FE00000C1103509F4F9C0173509F4F6C0F9C08D
:100FF0008091BD05813019F40091E70501C000E042
:1010000093FF29C081E40E94311F62E08091B60500
:101010000E94C3040E944C060023C1F08091E505A4
:10102000811105C060E87EEC82E090E0C2C08130B2
:1010300041F0E091BE05F091BF0586898460868B02
:10104000EDC060E87EE985E090E0B3C060E078E65E
:1010500081E090E0AEC094FF07C0C12C78E6D72EA7
:10106000EE24E394F12C07C060E1C62E68E6D62E8C
:10107000EE24E394F12C8330E1F2811111C088E178
:10108000849FF001859FF00D1124E45CFD4F82895F
:101090009389A489B589C816D906EA06FB0649F6DC
:1010A000011103C000E810E002C000E011E010925E
:1010B000BD05E091BE05F091BF05878980FDB9CFE0
:1010C000868986FDB6CF83FF03C0877F868B08C0E5
:1010D00081E40E94311F62E08091B6050E94C30442
:1010E00080E091E00E949A05E091BE05F091BF0575
:1010F000868984FF04C0812C912C54011CC050E1CE
:10110000852E912CA12CB12C16C0E1E0CE16DE0666
:10111000E104F10420F0C12CD12C7601D394960186
:10112000B501A40181E00E949D1A892B99F08C0CD5
:101130009D1CAE1CBF1CE091BE05F091BF05C2888E
:10114000D388E488F588C818D908EA08FB08E9F6C6
:1011500080E001C081E0E4EBF4E098012C543B4FC7
:101160009FEF9193E217F307E1F7882379F010924C
:10117000B4041092B504E091BE05F091BF058689D4
:101180008460868B81E091E00E94A92540E0B8014F
:10119000D8C693FF1FC081E40E94311F62E0809196
:1011A000B6050E94C3040E944C0660E078E082E02D
:1011B00090E00E943B0581113CCF1091B605E09173
:1011C000BE05F091BF05808991899093DF058093DA
:1011D000DE054AC727FF2DCF65CF62E00E94C3041A
:1011E00026C061E00E94C3048091DD059EEA980F4D
:1011F000923050F4E091BE05F091BF05968993FFBF
:1012000016C0833529F413C08E3489F08F3479F0F9
:101210008F3321F48091C205883249F480910F0206
:10122000882309F4C6C38EE40E94A305C2C381E4E7
:101230000E94311F8091700080FD0E94DF05809127
:10124000DD05803509F408C158F48E34B1F008F09A
:10125000A0C08F3311F00C9470118091C20529C386
:10126000833509F45DC2873509F4F6C0823511F083
:101270000C9470110E944C06EFC0E090BE05F090F7
:10128000BF05D70152964D905D906D907C9055971B
:1012900056968C9183FF0BC09091BD05913009F457
:1012A00072C0412C38E6532E66246394712CB82FFB
:1012B000B074BD8385FF03C000E011E002C000E808
:1012C00010E0C12EDD2480E090E053014201E0E80F
:1012D0008E2221EE35E03C832B831C013CE0230E63
:1012E000311CDC011196BF83AE830E94C83DEB81A7
:1012F000FC818193FC83EB838E819F8128163906C4
:1013000081F7FD81F11113C08091E9059091EA0503
:10131000A091EB05B091EC0588159905AA05BB05D0
:1013200031F48091E70590E08C159D0561F1C101D4
:101330002091E105213069F6C092E7050093E805A8
:101340002D81222341F03DE2430E34EB531E611CFC
:10135000711C0DE710E0D70156968C9185FF06C0F1
:10136000B0E84B0EB1E05B1E611C711C980140E0BF
:1013700050E0C301B2010E94A8343093E3052093EA
:10138000E4054093E50540E06CE070E081EE95E017
:10139000DAC56CE070E081EE95E00E94931F811148
:1013A0009FC70091BE051091BF05D8015696EC91DC
:1013B0005697F091E705E3FF09C0FF2311F0E062C3
:1013C00002C0EF7DD8015696EC9342C02091E5050E
:1013D000822F90E0A0E0B0E09C01AD012F5F3F4F75
:1013E0004F4F5F4FA091E105B0E00E940D359B018A
:1013F000AC01A091E305B0E0BA2FAA278091E405E3
:10140000A80FB11D0E9418359B01AC01AF2FB0E0B1
:10141000BA2FAA278091E805A80FB11D0E941835A0
:10142000E4FD04C0605F7F4F8F4F9F4FE5FF04C016
:101430006058714081099109F80102891389248952
:101440003589601771078207930711F083E001C0A7
:1014500081E08093BD0523C780E890E09A8389836B
:101460001092BD05C090DE05D090DF05C114D104F7
:1014700009F452C1E091BE05F091BF05E689E6FD91
:1014800073C0E1FF15C090910E028091B6059817C8
:1014900031F00E949F2F8091B60580930E0242E0AA
:1014A00051E0BE016F5F7F4FC6010E9419303DC001
:1014B000F4E0CF16D10458F421E0C21AD108D69432
:1014C000DC2CCC24D794C794E12CF12C1CC0E5FF74
:1014D00003C0A0E0B1E002C0A0E8B0E0BA83A983F5
:1014E000A60160E070E09A01AB0124503109410986
:1014F00051090E940D356B017C0130E8C30E31E0CB
:10150000D31EE11CF11CE4FD05C080E1C80ED11C16
:10151000E11CF11C8091DD0529813A81823549F475
:10152000B701A60180E00E949D1A892B09F4F4C03E
:10153000F0C0B90184EB94E00E94931F8111D0C6E2
:101540000E944C06E091BE05F091BF05878980FDA1
:10155000E3C029813A81B701A60181E00E949D1A6A
:10156000892B09F4D9C09BC68091DD05823551F0E5
:1015700060E870E084EB94E00E94931F882309F4F4
:10158000CBC0AEC680E890E00E949A0594E0C916F0
:10159000D104F0F0E090BE05F090BF05F70182891C
:1015A0009389A489B589BC01CD0164587F4F8F4FC1
:1015B0009F4F2DE730E040E050E00E94A834490101
:1015C0005A018901F8E6CF16F1E0DF0629F574C06B
:1015D000C6019695982F88279795879583519040B7
:1015E0002091C30577E0972E920E04EB14E07C0166
:1015F00020E8E20EF11C5C013FEFA31AB30A0E943F
:10160000C83D873009F4892DD8018D938D01C5011E
:10161000AE14BF0481F7BECFB9E6CB16B1E0DB064E
:1016200009F04FC060E0F701808991890E94951808
:10163000A4EBB4E080E090E030E22D914FEB420F5C
:101640004A3120F040ED420F4A3030F4E82FF0E00C
:10165000EC54FB4F20838F5F973011F09A3049F4A0
:10166000981738F0E82FF0E0EC54FB4F30838F5F91
:10167000F7CF9F5F9B3009F7EFEBF4E08291858312
:1016800024E0E43BF207D1F7E4ECF4E084E395E0F6
:101690008E179F0711F01192FBCF003932E013072C
:1016A00010F086E401C082E48093B40481E791E005
:1016B0009093B8048093B7049092B6048092B504D6
:1016C00024C081E7C81681E0D806F8F09601ADE79E
:1016D000B0E00E94F734AB01BC014D52544B61099C
:1016E00071092DE730E080E00E949D1A8D37910549
:1016F00020F096012F5F3F4F02C020E030E0309392
:101700003105209332058093330580E890E09A8379
:10171000898369817A8114C469817A8141E011C425
:1017200090910D02911190E19093B404E091BE0567
:10173000F091BF05868987FF03C090689093B40439
:1017400085FF05C09091B40490629093B40482FF29
:1017500007C09091B40494609093B4048B7F868BFF
:10176000878980FF05C08091B40488608093B404A9
:10177000809102018093B50480EE8093B6041092AC
:10178000B704ADC081E40E94311FE091DD05EB3D5F
:1017900009F48AC01F7088EF95E09093BF0580938D
:1017A000BE058E2F90E0FC01E05CF109E034F1050C
:1017B00008F085C5EC5CFF4F0C94E93400E010E0C4
:1017C000B2C280E091E00E949A058091DE0590917E
:1017D000DF0500EC14E06C01A5E1CA0ED11C7C0110
:1017E000BFEFEB1AFB0A60E00E9495188823D9F03E
:1017F000EC14FD0429F48091B404F801808313C033
:10180000A4EBB4E0C8010B96F8012D912193E817E1
:10181000F907D9F78091B805D8011B968C93045F1E
:101820001F4FC701DCCFE4EBF4E084858193B5E082
:10183000E53AFB07D1F740E061EF70E082C38091A9
:10184000DE058A3F08F03BC58093C2051092C105B2
:10185000EFE7FCE03197F1F700C0000083E40E945D
:10186000311F5FCB8091DE058093C30518C583E2ED
:1018700092E0A4EBB4E04DEC54E0FC012191CF01E7
:101880002D93F4E0AD3CBF07C1F7A8EFB5E085EEBE
:1018900094E02D91FA012193AF018E179F07C9F7AC
:1018A00040E061E370E04DC3E091BE05F091BF05FB
:1018B00086898093B40440E061E070E042C36091A7
:1018C000DE057091DF0580E090E00E9410176093C4
:1018D000B4047093B5048093B6049093B70440E0C9
:1018E00064E070E02EC364E070E084EB94E00E945A
:1018F000931F8111F5C46091B4047091B504809177
:10190000B6049091B7046093C4057093C5058093A5
:10191000C6059093C7050E94DE16C1C46091C40538
:101920007091C5058091C6059091C7050E94DE168D
:101930008FE79CE00197F1F700C0000083E40E946C
:10194000311FAFE7BCE01197F1F700C0000060E085
:1019500072E084EB92E00E94091F182F60E072E0B1
:1019600084EB92E00E94381F812FB8C46091C405B7
:101970007091C5058091C6059091C7050E94DE163D
:1019800040E260E072E084EB92E00E944C1FEFE9DD
:10199000FFE03197F1F700C00000882361F060910B
:1019A000C4057091C5058091C6059091C7050E9438
:1019B000DE168EE493C481E40E94311F80E00E9411
:1019C0009E1681117CC46BC46091DE05662309F408
:1019D00066C4E9EEF1E0A4EBB4E080E094919D935D
:1019E0008F5F31966813FACFAAC20E94D5168091F4
:1019F000DE05882319F00E94B9065FC48FE79CE0DA
:101A00000197F1F700C0000083E40E94311F0C949D
:101A100000009091DE05953008F051C4A8E19A9F2E
:101A2000F0011124E45CFD4F868983FD02C08E7FA6
:101A300001C0867F868BE0914001F09141010280D8
:101A4000F381E02DB4E19B9FE00DF11D1124859100
:101A500094914CE050E064EF70E003960E94C3372D
:101A60008091C0055BC2E091DE05E53008F027C437
:101A700028E1E29FF0011124E45CFD4F868980FD9E
:101A800008C08EE090E00E949A0540E06EE070E0B1
:101A900058C2F093BF05E093BE0584819581A6816D
:101AA000B7818093FC059093FD05A093FE05B0934C
:101AB000FF05908981899093DE058093DF0560E0C2
:101AC0008091DE059091DF050E949518082F3CC09B
:101AD0006BE070E08DEE95E00E94931F811100C4D1
:101AE0008091DF05882309F4DAC31091DE05812F88
:101AF000806F8093DD051092DF051092DE05E09087
:101B0000DE05F090DF058091DD05803F08F0B5C16E
:101B100060E0C7010E949518882309F4F2C1EDEE38
:101B2000F5E0A4EBB4E081918111C1C1119635E0DB
:101B3000E83FF307C1F78091DD05803F08F0BCC1A5
:101B400083EE8093DD0501E02091B8052093BF046A
:101B50008091DD05833E61F4E091BE05F091BF0503
:101B6000808991899093C1048093C0041EE0A7C02E
:101B7000853E09F0A3C0A091BE05B091BF05529665
:101B80004D915D916D917C9155974093C004509318
:101B9000C1046093C2047093C3048091B905D090CE
:101BA000BA058093C404D092C5048091BB0590917E
:101BB000BC059093C7048093C604E8ECF4E086EE7D
:101BC00094E030E231938E179F07E1F752966D91C2
:101BD0007D918D919C915597287119F420E3209364
:101BE000D10444EBE42E44E0F42E1AE05AE0852EB2
:101BF000912CA12CB12C611571058105910551F035
:101C0000A50194010E94A8346063D7015D966C938E
:101C1000B901CA011150B1E0EB1AF1081111EBCF73
:101C20008DE28093D7048093DA048AE38093E00402
:101C30008093E3048D2D869590E08454984F64E65C
:101C400070E00E948034962F182F6FE1892F0E9438
:101C50008E0561E2812F0E948E058091B9059091D9
:101C6000BA0525E0969587952A95E1F764E28F708D
:101C70000E948E058091B90567E28F710E948E05E2
:101C80008091BC056AE28695869586950E948E05B0
:101C90008091BB059091BC0535E0969587953A9566
:101CA000E1F76DE28F730E948E058091BB058F7105
:101CB00060E3880F0E948E0512E301C01CE0011151
:101CC00004C082E390E00E949A05612F38C161E070
:101CD0008091DE059091DF050E949518811106C064
:101CE00080E090E0FC01EC54FB4F09C0E4EBF4E031
:101CF00080E090E0019621912111FCCFF3CFCF013C
:101D0000845B94408F3F910509F010F41192F7CF56
:101D10008091DD05865E60E071E002C07595679593
:101D20008A95E2F70DC160E0C8010E9495188823EA
:101D300019F00F5F1F4FF7CF1093B5040093B40451
:101D400040E062E070E0FDC08091DE0581508431AA
:101D500018F084E18093DE050091DE058090FC059B
:101D60009090FD05A090FE05B090FF0510E08FE279
:101D7000D82E60E080E090E00E949518E091BE05CA
:101D8000F091BF05882309F450C08091B80584FF05
:101D90004CC08091B4048E3209F047C08091B504E4
:101DA0008E3209F042C0011107C0A12FB0E0AC543F
:101DB000BB4F8FE38C9339C00150448055806680BF
:101DC000778080819181A281B38184839583A6836A
:101DD000B783E12CF12C60E0C7010E94951888239D
:101DE00041F2E091BE05F091BF0580819181A28111
:101DF000B381481659066A067B0699F41C50E12FF8
:101E0000F0E0DF01AC54BB4FDC92A4EBB4E0EB5448
:101E1000FB4FCF010B962D9121938E179F07D9F77A
:101E2000A8CFEFEFEE1AFE0AD6CF84829582A68263
:101E3000B782812F90E0DC01AC54BB4F119520E0BC
:101E40003D91E22FF0E0EC54FB4F30832F5F2113E4
:101E5000F7CF8195811103C01092B40481E0E82F7F
:101E6000F0E0EC54FB4F10828F5FC9F76091DE0504
:101E7000FCE06F9FB001112463C0153008F048CE1C
:101E800028E1129FF0011124E45CFD4FF093BF059F
:101E9000E093BE058091FC059091FD05A091FE05A3
:101EA000B091FF0584839583A683B78331CE9C913F
:101EB000891709F43BCE21C01530D0F488E1189F72
:101EC000F0011124E45CFD4FF093BF05E093BE05E3
:101ED0008091FC059091FD05A091FE05B091FF0554
:101EE00084839583A683B78360E0C7010E94951819
:101EF000F092DF05E092DE05B7C09FEFE91AF90A1C
:101F000007CE8091DD05803F08F0D9C1BACD809120
:101F1000DE05853008F081E08093C0050E94FD0455
:101F2000BEC16091DE05E091DF05F0E0E054FA4FBC
:101F3000A4EBB4E0862F91919D938150E1F770E07E
:101F400040E084EB94E00E94C91FCAC160E080E0D9
:101F500090E00E949518811116C08091DE058823BB
:101F600009F49DC1E091BE05F091BF058091380252
:101F700090913902A0913A02B0913B0284839583FB
:101F8000A683B7837ECD8091B80584FFE6CF80918C
:101F9000B4048E3211F78091B5048E32F1F6E091DF
:101FA000BE05F091BF05C480D580E680F7808081B2
:101FB0009181A281B38184839583A683B783809125
:101FC000DE05882351F200E010E060E0C8010E94C5
:101FD0009518882311F2E091BE05F091BF0580812C
:101FE0009181A281B381C816D906EA06FB0609F4DD
:101FF000A7CD0F5F1F4FE9CF809138029091390232
:10200000A0913A02B0913B028093FC059093FD05AC
:10201000A093FE05B093FF0560E080E090E00E9491
:1020200095183DC11530B0F4A8E11A9FF0011124B4
:10203000E45CFD4FF093BF05E093BE058091FC0585
:102040009091FD05A091FE05B091FF0584839583D5
:10205000A683B78360E08091DE059091DF050E9442
:102060009518882309F42BC19091B805E091BE051D
:10207000F091BF0594FF09C080819181A281B38155
:1020800084839583A683B78301C140815181628196
:1020900073814087518762877387148615861686F9
:1020A000178686898870868B90FD02C0178A02C0C9
:1020B00081E0878B8091BC04813409F049C0809114
:1020C000BD04843509F0B1C08091BE04823509F0A9
:1020D000A1C020E130E040E050E0BA0180E00E9481
:1020E0009D1AE090BE05F090BF05F7018689982FF4
:1020F0009160968B2091B8049091B904922B913005
:1021000011F48162868BF70182899389A489B5894C
:10211000BC01CD016051710981099109D688D5FEB4
:1021200005C020E031E040E050E004C020E830E0AD
:1021300040E050E00E94A834213D32404105510565
:1021400008F47AC08D2D8068D70156968C9374C0A0
:10215000883559F48091BD04863409F066C08091B9
:10216000BE04843409F061C01AC0833459F48091EC
:10217000BD04813409F059C08091BE04833509F053
:1021800054C00DC0823409F050C08091BD04893420
:1021900009F04BC08091BE048E3409F046C024E0A3
:1021A00030E040E050E0BA0180E00E949D1A80914A
:1021B000B404863469F48091B504853579F480914E
:1021C000B6048A3459F48091B704893439F42DC0A7
:1021D0008F3F21F48091B5048F3F39F1E091BE0526
:1021E000F091BF058689982F9161968B428953891A
:1021F000648975894130B8E65B07B1E06B0771050A
:10220000D8F0413058406240710510F4816913C024
:10221000816311C0883549F40E949F2FE091BE056B
:10222000F091BF058689836006C0E091BE05F091FC
:10223000BF058689816C868B8FEF810F843030F5E6
:1022400060E08091DE059091DF050E94951884EB97
:1022500094E00E949720E0914001F09141010280BA
:10226000F381E02D34E1139FE00DF11D11248591E0
:1022700094914CE050E064EB74E003960E94D237F6
:1022800080912102811102C00E941B23E091BE05B2
:10229000F091BF05868983FF02C00C94500880919D
:1022A0000F02882321F083E40E94A30506C08FE774
:1022B0009CE00197F1F700C0000083E40FC080911B
:1022C0000F02882321F085E40E94A30506C0AFE732
:1022D000BCE01197F1F700C0000085E40E94311FB7
:1022E0002796E2E10C943C35A4E0B0E0EAE7F1E1A6
:1022F0000C942035459A3D9882E08093680080E2F6
:1023000080936C0080B7846880BF8FE080937E00EC
:1023100083B5816083BD84E79BEC909389008093B3
:10232000880080916F00826080936F001092C105D9
:102330001092C3051092C0051092B6051092BD050B
:1023400080E690E00E94C83D8093C2050E94552718
:10235000E0914001F09141010190F081E02D09955B
:1023600080913F0182FF03C081E08093C00588E631
:1023700090E00E94181F61E08091B6050E94C3049E
:102380000E9430152FEF31EE44E0215030404040A4
:10239000E1F700C000000E9476158823E1F11F924A
:1023A0008F9385E891E09F938F9384EB94E09F93C4
:1023B0008F930E94E13784EB94E00E947F26809106
:1023C000BB028F938091BA028F938091B9028F9351
:1023D0008091B8028F938091B7028F938091B6025B
:1023E0008F938091B5028F938091B4028F9387E78A
:1023F00091E09F938F9324EB34E03F932F930E94BF
:10240000E13784EB94E00E947F260FB6F894DEBF9C
:102410000FBECDBF7AC08DB581608DBD8CB58D7F6F
:102420008CBD8CB58E7F8CBD1092520210926A02C8
:102430001092820210929A021092B2020E944217E7
:102440008823B9F01F928F9384E691E09F938F9336
:1024500084EB94E09F938F930E94E13784EB94E0A8
:102460000E947F260F900F900F900F900F900F906B
:102470004CC089E08093210266E9E62E61E0F62EE9
:1024800091E09B83C7010E94D03D6093FC0570934F
:10249000FD058093FE059093FF056F3F7F4F8F4FA3
:1024A0009F4F89F0C70104960E94D63D9093DF05A7
:1024B0008093DE058B81806F8093DD05F1E7F093DB
:1024C000DC050E9448072B812F5F2B8336E0E30E4B
:1024D000F11C2530B9F6109221020E941B23809135
:1024E000380290913902A0913A02B0913B02809358
:1024F000FC059093FD05A093FE05B093FF050E9497
:10250000B9068091C0050E94FD0460E08091B60587
:102510000E94C3047894612C712C44EB54E05C83DA
:102520004B83212C312C210158E1852E0E941C2E39
:10253000882309F45AC18091700080FF03C00E9473
:10254000DF053EC10E942A28009709F446C1109277
:102550002406FC017096259134913C832B833A83A9
:102560002983FC01C590D4907601F89448EF55E09A
:102570005093BF054093BE0520912102211116C042
:10258000F6012081243491F4E0914001F091410161
:1025900022813381AC01421B530B9A01359527955B
:1025A000359527955DEC259F902C1124FC017296A2
:1025B00025913491F90109958C0178948091C00599
:1025C000981679F0EB81FC81808182FF0AC090929D
:1025D000C005911002C00E94B9068091C0050E94FA
:1025E000FD04F60180818E33A9F4899CF001112449
:1025F000E45CFD4F008911890F5F1F4F8481958135
:10260000A681B781E091BE05F091BF0584839583D3
:10261000A683B78301151105F9F0F8940F3FFFEF7A
:102620001F0731F422EE2093DD059092DE050EC0E7
:10263000899CF0011124E45CFD4F168A892D806F7E
:102640008093DD051093DF050093DE0531E73093BD
:10265000DC050E944807789480912102811128C0EE
:10266000F60180818E3421F58091C005882301F127
:10267000889EF0011124E45CFD4F96899860968B4A
:10268000E0914001F09141010280F381E02D24E1CD
:10269000829FE00DF11D1124E590F4904CE050E094
:1026A00067E571E0C70103960E94C3370E941B23B0
:1026B00080912102833009F073C0F7018081833556
:1026C00009F073C0E0914001F09141010188F28965
:1026D000E02DB496A591B4918091B70580FD03C01B
:1026E0008C9182FF21C08091B7058E7F8093B705C2
:1026F000EB81FC8180818B7F80838C918B7F8C939D
:1027000029E4E22E21E0F22E0AE812E520EE3FEF66
:1027100042E064E870E083E290E00E94502C0E9466
:102720001B23612C712C41C0E091BE05F091BF05C7
:1027300080819181A281B38180879187A287B387AD
:102740000E941C338091B70581608093B705EB81AF
:10275000FC8180818460808399E3E92E91E0F92EE9
:102760000AE812E520EE3FEF42E064E870E083E221
:1027700090E00E94502C0E941B238091B70581FDA0
:1027800019C0FAEA26EE36E941E0F1502040304027
:102790004040D9F7000084EB94E09C838B830EC00B
:1027A000E4EBF4E0FC83EB8309C024EB34E03C83EE
:1027B0002B8304C044EB54E05C834B8300E21EE4B3
:1027C0000E941C2E8111FCCF5FEF80E792E05150F8
:1027D00080409040E1F700C0000010920902109282
:1027E0000A0210920B0210920C028091B70580FF32
:1027F00024C0F8948091B70581FF04C0C3010E94F2
:102800004F3303C0C3010E9464323C01892B21F085
:102810008091B70580FD10C088E690E00E94181FE7
:102820008091B7058E7F8093B705E981FA81808119
:102830008B7F80830E941B23789480913F0181FFCE
:102840005AC080912102813009F055C0F0902406D1
:10285000FF2009F450C00032FEE41F0709F049C010
:1028600023E12F1518F01092240602C083E1F82E00
:1028700040913B0150913C0141505109A12CB12C98
:10288000C12CD12CE12C01E02AE130E06AE070E0BB
:1028900085E090E00E94AB2ACF2CEB80FC8000E02A
:1028A00010E020EE3FEF42E06AE070E085E090E06B
:1028B0000E94982C4B815C8184E0443B580769F06E
:1028C000FA0101900020E9F7CF014497841795079A
:1028D00039F4E3EBF4E0FC83EB8302E21EE402C094
:1028E00000E010E02B813C812F5F3F4F3C832B8326
:1028F00002C00E5F1F4F31EA231630EF330639E175
:102900004306510430F00E94D516212C312C2101B0
:1029100005C04FEF241A340A440A540A80913F013B
:1029200084FF04CE80912102811100CE80910902A2
:1029300090910A02A0910B02B0910C02813854E8E8
:1029400095075EE1A507B10538F08091700081110F
:10295000EDCD0E94D005EACD0196A11DB11D809359
:10296000090290930A02A0930B02B0930C02DECDF1
:102970001F920F920FB60F9211242F933F934F93F4
:102980005F936F937F938F939F93AF93BF93EF93D7
:10299000FF93359929C08091000190910101909396
:1029A000BF058093BE05109224061092DD050E949B
:1029B000480760E08091B6050E94C3048091BE057F
:1029C0009091BF05909301018093000188EF95E0FD
:1029D0009093BF058093BE051092090210920A02DF
:1029E00010920B0210920C02FF91EF91BF91AF91E8
:1029F0009F918F917F916F915F914F913F912F9117
:102A00000F900FBE0F901F9018952A9A229A2D9A18
:102A1000259A2498239A8DB58E7F8DBD83E58CBD34
:102A20008DB508958EBD0DB407FEFDCF8EB508950A
:102A30008FEF0E9412150895FB01E40FF51F39E096
:102A40006E177F0761F0229198E0880F482F422788
:102A500047FD8327220F9150C1F78F77F1CF08955B
:102A60000E9405150895A5E0B0E0E9E3F5E10C94B6
:102A70002F354A835B836C837D83806489830E94C6
:102A800012158D810E9412158C810E9412158B8166
:102A90000E9412158A810E94121541E050E0BE0189
:102AA0006F5F7F4F80E00E941C1544E050E0BE0144
:102AB0006E5F7F4F0E941C15880F81600E94121567
:102AC0001FEF0E941815115011F087FDFACF2596BF
:102AD000E3E00C944B35CF932A980E943315C82F0E
:102AE0002A9A0E9418158C2FCF910895EF92FF9289
:102AF0000F931F93CF93DF938FEF9FEFDC018093B2
:102B0000110690931206A0931306B0931406109228
:102B10001506809110068E7F80931006CAE00E94F1
:102B20001815C150E1F7DAE040E050E0BA0180E06A
:102B30000E946B15813031F0D150B1F78093B4020F
:102B4000C1E091C084EBE82E82E0F82E1AE02A98CA
:102B50004AEA51E060E070E088E00E943315D82F27
:102B60008130C1F4870184E0E80EF11C0E94181541
:102B7000F80181938F01EE16FF06C1F78091B6022E
:102B8000813031F48091B70210E08A3A11F402C02A
:102B900010E0D6E02A9A0E9418158D2F8B7F813085
:102BA00061F08FEF810F112311F0182FD0CFD630A5
:102BB00020F0F701D083C2E056C00FEF13E040E0F1
:102BC00050E0BA0187E30E946B15D82F8230A8F538
:102BD00040E050E060E070E489E20E946B158111F2
:102BE00027C02A9840E050E0BA018AE30E943315DA
:102BF000D82F0E9418158093B8020E941815809350
:102C0000B9020E9418158093BA020E941815809389
:102C1000BB022A9A0E9418158091B80286FB882769
:102C200080F99091100680FB90F99093100605C0F2
:102C30000150110921F6C3E016C0D53041F440E03F
:102C400050E0BA0181E00E946B1581110BC040E099
:102C500052E060E070E080E10E946B15882319F07B
:102C6000C5E001C0C4E08C2FCDB7DEB7E6E00C9420
:102C70004835CF93DF93AB01BC012A9880911006B1
:102C800080FD07C089E0440F551F661F771F8A9596
:102C9000D1F781E10E943315811115C00E941815EA
:102CA0008E3FE1F7C4EBD2E00E941815899384E0CF
:102CB000C43BD807C9F70E9418150E9418152A9A14
:102CC0000E94181580E0DF91CF910895CF93DF9394
:102CD000AB01BC012A988091100680FD07C089E0F5
:102CE000440F551F661F771F8A95D1F788E10E9410
:102CF0003315811120C00E9418158EEF0E94121505
:102D0000C4EBD2E089910E94121584E0C43BD8073D
:102D1000C9F70E9418150E9418150E941815982FBF
:102D20009F71953041F40E9418158823E1F32A9A87
:102D30000E94181580E0DF91CF9108950F931F93A3
:102D4000CF93C82F00E018EF21E043E050E065E0AA
:102D500070E08FE090E00E94002BCC23F1F0C0E106
:102D600060911106709112068091130690911406DD
:102D70000E946616882319F0C15091F7FFCF109278
:102D8000150600E010E021E043E050E065E070E06F
:102D90008FE090E00E94002B03C081E08093150635
:102DA00080E0CF911F910F9108958091150688239F
:102DB00021F081E00E949E16FACF0895CF92DF9213
:102DC000EF92FF92CF93C0901106D0901206E09040
:102DD0001306F0901406C616D706E806F90611F495
:102DE0008FEF18C06B017C010E94D516C0E0C701AF
:102DF000B6010E943916C150882319F0C111F7CFCE
:102E0000EFCFC0921106D0921206E0921306F09214
:102E1000140680E0CF91FF90EF90DF90CF9008955F
:102E2000CF92DF92EF92FF92C0902F02D0903002AB
:102E3000E0903102F0903202611571058105910533
:102E400069F48091330290913402A7019601281B06
:102E5000390B41095109CA01B9010FC09B01AC01ED
:102E60002250310941095109A0913702B0E00E9476
:102E70000D356C0D7D1D8E1D9F1DFF90EF90DF9019
:102E8000CF900895A0E0B0E0E8E4F7E10C9422359B
:102E900060E070E0CB010E94DE168111E8C0D091A5
:102EA000760480907A0490907B04A0907C04B0908B
:102EB0007D04C501B4010E94DE16C82F8111D9C05E
:102EC000E091C502F091C60284E0F695E7958A95F7
:102ED000E1F7F0933402E09333028091CA029091BB
:102EE000CB02009719F0A0E0B0E008C08091D802B2
:102EF0009091D902A091DA02B091DB0280932B026B
:102F000090932C02A0932D02B0932E02C090C20287
:102F1000D090C302E12CF12CA091C40220912B028D
:102F200030912C0240912D0250912E02B0E00E946F
:102F30000D352B013C01B501A4014C0D5D1D6E1D2D
:102F40007F1D8F0120E030E0D301C201840F951F67
:102F5000A61FB71F800F911FA21FB31F80932F02C0
:102F600090933002A0933102B09332028091C70255
:102F70009091C802009719F0A0E0B0E008C08091DD
:102F8000D4029091D502A091D602B091D7028419B3
:102F90009509A609B7098C199D09AE09BF09801BBF
:102FA000910BA20BB30B8093230290932402A09366
:102FB0002502B09326028091C1028093370280914E
:102FC000BF029091C00290933602809335024093E5
:102FD0002702509328026093290270932A028FEFF0
:102FE0009FEFDC018093160690931706A0931806B6
:102FF000B0931906DD3038F4DB3098F4D43029F082
:10300000D630C9F502C0DE30B1F5E091BE05F091D1
:10301000BF051482158216821782809110068D7F5B
:1030200013C08091E0029091E102A091E202B09180
:10303000E302E091BE05F091BF0584839583A683EA
:10304000B78380911006826080931006E091BE05E0
:10305000F091BF0584819581A681B7818093380264
:1030600090933902A0933A02B0933B0205C0C1E0AD
:1030700003C0C2E001C0C3E08C2FCDB7DEB7E0E1F2
:103080000C943E358F929F92AF92BF92CF92DF9277
:10309000EF92FF922091100621FF0EC042E0660FD2
:1030A000771F881F991F4A95D1F7CC24CA94DC2C2E
:1030B000EC2C5FE0F52E09C0660F771F881F991F63
:1030C000CC24CA94DC2CE12CF12C209135023091D7
:1030D000360240E050E00E94A8344B015C01809130
:1030E000270290912802A0912902B0912A02BC01E6
:1030F000CD01620F731F841F951F0E94DE16F4011D
:10310000EC54FD4F80819181A281B381BC01CD013E
:103110006C217D218E219F21FF90EF90DF90CF9039
:10312000BF90AF909F908F900895AAE0B0E0EBE938
:10313000F8E10C9420351C016A83E091BE05F09102
:10314000BF05C480D580E680F780809116069091F7
:103150001706A0911806B0911906C816D906EA06F6
:10316000FB0651F0C0921606D0921706E0921806A0
:10317000F092190610921A0680911A06882389F097
:1031800020911A0230911B023E832D8322153305B4
:1031900098F02215330529F4813019F43A8133234C
:1031A00059F0C701B6010E9410172B013C0110E035
:1031B0001E821D82198240C000911002809016026A
:1031C00090901702A0901802B0901902C0901102BE
:1031D000D0901202E0901302F090140210911502A8
:1031E0001982240135018FEF481A580A680A780AB3
:1031F000C501B4010E94DE1690E2099FF00111247E
:10320000EC54FD4F4081442309F4E9C0453EC9F424
:10321000B0960F5F0031B1F7C114D104E104F1049D
:1032200009F0CCC0812F90E020913302309134021C
:103230008217930708F0BBC01F5F5301420100E0F3
:10324000D0CF83858F3009F053C0AA81AA2301F320
:10325000842F90E001978F709927BDE0B89FB0014F
:10326000B99F700D11246C547B4F9F017A87698739
:10327000CF010A969C838B83F887EF83AF81B88553
:1032800011965C91A985BA855D93BA87A9878F81CC
:103290009885029698878F83AB81BC818A179B079C
:1032A00069F7CB0105969C838B83CF010C96D901DE
:1032B0001E965C91AB81BC815D93BC83AB832E5F1A
:1032C0003F4F8217930799F7848DDB011B968C93F0
:1032D0001B97868D1C968C931C9746FF02C01D96EB
:1032E0001C924F70413009F093CF31E0398390CF79
:1032F000B981BB2361F02D813E812215330509F48C
:1033000070C02F5F3F4F3E832D83198281CF4E3295
:1033100029F49181903211F484FD7ACF83FD78CF26
:103320008D819E8182159305D9F5CF0164EB74E000
:10333000AB01DC012D91CD01DA012D93AD01B4E09B
:103340004F3B5B07B1F71092BF042A81222309F497
:103350004AC01092C0048091BE048093BF04809143
:10336000BD048093BE048091BC048093BD04809111
:10337000B4048E3219F08EE28093BC0424EB34E066
:10338000DB018D91BD01803221F0D9018C932F5F3B
:103390003F4FDB018C918111F3CFD9011C9223C0E7
:1033A0002D813E812F5F3F4F3E832D8331CF909102
:1033B0001006892F827091FD3FCF6EC08091370239
:1033C000181708F439CFC701B6010E9442186B01E3
:1033D0007C010E9410172B013C0110E02DCF80E0F2
:1033E00005C082E003C03E822D8281E0A091BE052F
:1033F000B091BF054489558960E070E0BA01552756
:103400004427228D338D2901612C712C44295529A3
:10341000662977294D935D936D937C93139751960D
:103420003C922E925097448D558D668D778D529695
:103430004D935D936D937C93559793859093B805C9
:10344000268937893093BC052093BB05208D318DAB
:103450003093BA052093B9058823E9F0AD81BE8188
:10346000B0931B02A0931A020093100280921602DE
:1034700090921702A0921802B0921902C092110203
:10348000D0921202E0921302F092140210931502ED
:1034900080931A0601C080E02A96E2E10C943C3544
:1034A000A0E0B0E0E6E5FAE10C942A356B017C017E
:1034B000E091BE05F091BF0584859585A685B78509
:1034C000C816D906EA06FB0660F480819181A281C4
:1034D000B38180879187A287B38714861586168665
:1034E0001786C091BE05D091BF050C851D852E8520
:1034F0003F85688579858A859B85C016D106E20659
:10350000F306B1F00E944218688779878A879B8703
:10351000E091BE05F091BF0584859585A685B785A8
:103520000196A11DB11D84879587A687B787D9CF3E
:10353000CDB7DEB7E8E00C944635A9E0B0E0E3EAA9
:10354000FAE10C942035E091BE05F091BF05428868
:10355000538864887588441555056605770518F005
:1035600080E090E0E2C019016A017B018D83209127
:103570003702A0913502B0913602AD0160E070E0F3
:103580004E835F836887798730E00E94F7344B0170
:103590005C01C301B2016C197D098E099F09698321
:1035A0007A838B839C83C701B601A50194010E9495
:1035B000A83429013A01A5019401C301B2010E9476
:1035C0006434C61AD70AE80AF90AC701B6012E817F
:1035D0003F81488559850E94A83449015A012E81AE
:1035E0003F8148855985C501B4010E946434C61ADB
:1035F000D70AE80AF90AC301B2010E94501AE09101
:10360000BE05F091BF0560857185828593850E9416
:103610001017680D791D8A1D9B1D0E94DE1604EB94
:1036200014E01F821E828E819F818215930509F40A
:103630004BC08091350290913602A0E0B0E0C816F0
:10364000D906EA06FB06C0F17D817130E1F08FEF0B
:10365000881A980AA80AB80A8091370290E0A0E078
:10366000B0E088169906AA06BB0698F09FEF491AA3
:10367000590A690A790AC301B2010E94501A812CC1
:10368000912C540106C080E00E949E168823F9F216
:1036900067CFE091BE05F091BF0560857185828599
:1036A00093850E941017680D791D8A1D9B1D0E942D
:1036B000DE16C12CD12C760149815A816B817C8127
:1036C000452B462B472B21F45D81513061F526C0F7
:1036D000F601EC54FD4F6D81613019F4D8018C91E5
:1036E00002C08081F801808349815A816B817C818D
:1036F000415051096109710949835A836B837C8365
:103700006E817F816F5F7F4F7F836E837FEFC71AEC
:10371000D70AE70AF70A0F5F1F4F85CF80E00E94A4
:103720009E1681111DCF8E819F812996E2E10C9416
:103730003C35AAE1B0E0EFE9FBE10C9420359C8731
:103740008B87788F6F8BDC018D909D90AD90BC90B6
:10375000BFEF8B1A9B0AAB0ABB0A80911006209020
:1037600035023090360281FF11C03694279436948A
:1037700027942FEF3FEF4FEF5FE02F833887498784
:103780005A8744E050E05E834D830EC03694279400
:103790008FEF9FEFA0E0B0E08F839887A987BA876B
:1037A000A2E0B0E0BE83AD836101E12CF12CC50144
:1037B000B401A70196010E94A83429013A01A7018A
:1037C0009601C301B2010E94643469837A838B83BA
:1037D0009C838091270290912802A0912902B091A8
:1037E0002A02480E591E6A1E7B1E409127025091E4
:1037F00028026091290270912A0280912B029091F7
:103800002C02A0912D02B0912E02840F951FA61FAD
:10381000B71F481659066A067B0608F0C4C0C301E4
:10382000B2010E94DE16C501B401A70196010E94F3
:10383000A8347A8F698F8090270290902802A090F8
:103840002902B0902A0200912B0210912C022091A3
:103850002D0230912E02800E911EA21EB31EA501D4
:10386000940121503109410951092D873E874F8725
:10387000588B2091230230912402409125025091CF
:103880002602298B3A8B4B8B5C8B80903702912CD4
:10389000A12CB12CAD81BE81A69FA001A79F500D88
:1038A000B69F500D11245E8B4D8B00E010E0498DCA
:1038B0005A8D4215530508F061C02D853E854F8510
:1038C00058894216530664067506E9F469897A89AF
:1038D0008B899C89A50194010E94A834CA01B90171
:1038E000A70196010E94A834DC01CB010196A11D1D
:1038F000B11DE98DFA8DAF0160E070E08417950786
:10390000A607B707D8F1ED89FE89E00FF11FEC5447
:10391000FD4F80819181A281B3812F8138854985B6
:103920005A8582239323A423B5234D815E81040FFE
:10393000151F892B8A2B8B2BD1F4C980DA80EB8061
:10394000FC80898D9A8DC80ED91EE11CF11CAB85B7
:10395000BC85CD92DD92ED92FC921397EF89F88DA4
:10396000408251826282738280E090E01EC0298D85
:103970003A8D2F5F3F4F3A8F298F99CF89819A8156
:10398000AB81BC818C0D9D1DAE1DBF1D89839A83AB
:10399000AB83BC839FEF491A590A690A790A812CC3
:1039A000912C540122CF81E090E06A96E2E10C94E0
:1039B0003C35A9E1B0E0EFEDFCE10C9420355C0171
:1039C0006A017B0120911602309117024091180282
:1039D000509119022E873F87488B598B0091100216
:1039E00010E00F5F1F4F0F7011270115110541F4F3
:1039F0002F5F3F4F4F4F5F4F2E873F87488B598B2D
:103A00008091100681FD0DC08FEF9FEFA0E0B0E028
:103A10008A8B9B8BAC8BBD8BA2E0B0E0BD87AC8763
:103A20000CC02FEF3FEF4FEF5FE02A8B3B8B4C8BAF
:103A30005D8B44E050E05D874C8719821A821B82BF
:103A40001C82BE016B5F7F4FCE0101960E94991BC5
:103A5000892B29F060E070E080E090E046C16E853F
:103A60007F85888999890E94DE1685E0000F111FE5
:103A70008A95E1F7C8018C549D4F9A87898789817F
:103A80009A81AB81BC81E985FA85B58BA48B938F34
:103A9000828F48E050E0B501CF010E94D23743E069
:103AA00050E06AE272E089859A8508960E94C337E1
:103AB000A985BA855C96CD92DD92ED92FC925F97D6
:103AC00080E21B968C9380E00E949E168111C2CFEB
:103AD00089809A80AB80BC80C501B4010E94101718
:103AE0006E8B7F8B888F998F2090350230903602B5
:103AF000B0913702BB87910140E050E0C701B601A9
:103B00000E94A834EB854E2E512C612C712CCA01D9
:103B1000B901A30192010E94A8348901FB85F29D9D
:103B20009001F39D300D112440E050E0C701B60133
:103B30000E94A834672B682B692B11F401501109DE
:103B4000C1016C857D850E9480349B0140E050E07E
:103B5000C501B4010E94A8348091270290912802E7
:103B6000A0912902B0912A02820F931FA41FB51FB2
:103B70008D839E83AF83B887612C712C1B862C8527
:103B80003D851901412C512C8091350290913602CE
:103B90006C857D850E9480349B0140E050E0698106
:103BA0007A818B819C810E94A8349B01AC01C20167
:103BB000B1010E9464346B017C018D809E80AF80D6
:103BC000B884BE016B5F7F4FCE0101960E94991BA6
:103BD000892B21F03B853F5F3B8783018D819E814F
:103BE000AF81B88588169906AA06BB0621F0C501E3
:103BF000B4010E94DE1680911006F601EC54FD4FD0
:103C000060167106A0F481FF0DC089819A81AB8195
:103C1000BC812A893B894C895D8982239323A42313
:103C2000B5230BC089819A81918380830FC081FF66
:103C300009C08A899B89AC89BD8980839183A283CD
:103C4000B38304C0AFEFBFEFB183A08380E00E94D5
:103C50009E1680912B0290912C02A0912D02B09182
:103C60002E02BC01CD01680D791D8A1D9B1D0E948D
:103C70006616BFEF6B1A7B0A0615170508F084CF8E
:103C8000EB85EE2331F16E857F85888999890E94C5
:103C9000DE16209137028091350290913602289FDE
:103CA000A001299F500D1124C8010196489F900141
:103CB000499F300D589F300D1124C901A0E0B0E09C
:103CC000E985FA85848F958FA68FB78F81E00E9452
:103CD0009E1680911A0290911B0260E001960E944C
:103CE00095186E897F89888D998D6996E2E10C948B
:103CF0003C35ABE0B0E0EFE7FEE10C9422351B86EB
:103D00001A86611571058105910521F460E070E066
:103D1000CB017BC0409137022091350230913602B1
:103D2000429FF001439FF00D11248F0120E030E00D
:103D3000980111270027061717072807390730F3BE
:103D40002B013C01E091BE05F091BF058091160664
:103D500090911706A0911806B09119068483958357
:103D6000A683B78380E090E000E010E04E012AE0F7
:103D7000820E911C22E2C22E22E0D22E34EBA32E20
:103D800034E0B32E7C012FEFE21AF20A60E00E94C9
:103D900095188823B1F09F928F92DF92CF92BF92B5
:103DA000AF920E9403388A859B850F900F900F90E9
:103DB0000F900F900F900817190708F48C01C70196
:103DC000E1CF81E0E816F10409F4A0CF0F5F1F4FA7
:103DD000003127E2120708F099CF1F930F9389E172
:103DE00092E09F938F938E010F5F1F4F1F930F934E
:103DF0000E94E137B301A201C8010E94D91C0F90B3
:103E00000F900F900F900F900F902B96E0E10C9475
:103E10003E35FC01680F791F80E0E617F70739F09F
:103E20009191980F981708F49F5F892FF6CF089506
:103E30002091C00025FFFCCF9093C5008093C40063
:103E400082E28093C00088E18093C10087E0809384
:103E5000C2008091C00087FF03C08091C600F9CFE7
:103E600008959091C00095FFFCCF8093C6000895FF
:103E70000F931F93CF93DF93EC018C01060F171F55
:103E8000C017D10721F089910E94311FF9CFDF912E
:103E9000CF911F910F910895CF92DF92EF92FF92F1
:103EA000CF93DF939B01FC0152EFC52E59E4D52E31
:103EB00052E0E52EF12C50E0A6B1A072B0E0A417BC
:103EC000B50711F5A1E0CA1AD108E108F108F1F02F
:103ED000A091C000A7FFF0CFA091C000D091C60074
:103EE000A4FD16C0CA2FC870A3FD14C0211531054A
:103EF00031F40E94091FD81771F0C0E80CC0D083BC
:103F0000215031093196D8CFC1E005C0C2E003C0CD
:103F1000C3E001C0C4E08C2FDF91CF91FF90EF9000
:103F2000DF90CF900895A1E0B0E0E9E9FFE10C94C3
:103F3000303540E20E944C1F89838FE99FE0019752
:103F4000F1F700C000008981882391F08EE40E947F
:103F5000311F80910F028823B9F08EE40E94A305DF
:103F60008981805D8983CE0101960E947F260CC0E5
:103F700081E40E94311F80910F02882331F081E497
:103F80000E94A30580E001C08FEF2196E2E00C942F
:103F90004C350F931F93CF93DF93EC018B018091EE
:103FA0000F02882351F0442321F085E40E94A305E9
:103FB0000CC083E40E94A3050AC08FE79CE0019730
:103FC000F1F700C00000442311F085E401C083E450
:103FD0000E94311F8FE193E00197F1F700C00000CC
:103FE000B801CE010E94381FB801CE010E94091FFE
:103FF0000E94311FDF91CF911F910F91089540963C
:10400000FC01A591B4918C9184608C9380E090E048
:10401000089581E080932102809320027894E091BA
:104020004001F09141010580F681E02D099580E085
:1040300090E0089580912102813051F480911E0218
:1040400090911F020A9790931F0280931E0204C052
:1040500010920F021092200210922102E091400172
:10406000F09141010190F081E02D099580E090E010
:1040700008951092210280911E0290911F020A97CA
:1040800090931F0280931E0280912002882339F0B2
:1040900083E0809321021092500110924F01809191
:1040A0002102E0914001F091410195E0899FE00DEE
:1040B000F11D11240190F081E02D099580914F01AF
:1040C00090915001089582E080932102E091400197
:1040D000F09141010284F385E02D099580E090E0A4
:1040E000089580E090E00895FC0180911B06909176
:1040F0001C06893C910568F081E080932102789448
:10410000E0914001F09141010580F681E02D099593
:1041100008C0889748F07096A591B4918C918460FE
:104120008C9380E090E008958FEF9FEF0895FC015D
:104130008285838781858287808581878EE28087DB
:1041400014860895EF92FF920F931F93CF93DF93FE
:1041500080911C0290911D02892B09F45AC060E0E5
:1041600080911E0290911F020E949518882309F4E5
:10417000C6C060E270E08FE090E00E94BC2C20910D
:104180001C0230911D0282E491E09F938F93C9013C
:104190000197EAE0F0E0BF010E9480346F5F7F4F3B
:1041A0007F936F9380911E0290911F02BF010E9426
:1041B00080346F5F7F4F7F936F933F932F9381E79F
:1041C00092E09F938F9384EB94E09F938F930E9450
:1041D000E13724EB34E040E050E06FEF7FEF81E027
:1041E0000E94ED2C6DE270E08FE090E00E94BC2C0C
:1041F000C0911E02D0911F028DB79EB70C960FB6CC
:10420000F8949EBF0FBE8DBF8FE0E82E85E0F82E9C
:1042100044C060E080911C0290911D020E9495189C
:10422000882309F49CCF80911C0290911D02019675
:1042300090931D0280931C02ECCF60E0CE010E949F
:104240009518882309F44DC08091B8052091BC04CD
:1042500084FD3AC08EEE94E0FC013491231731F1D5
:104260000396E816F906C1F70DE71FEE203291F12B
:1042700084EB94E00E94972080914F01909150012F
:1042800024EB34E04AE852E5C817D90741F560EF5E
:104290007FEF82E00E94ED2C219680911E0290918A
:1042A0001F020A96C817D90740F225C03196E4913B
:1042B0003091BD043E13D4CFFC013296E49130918D
:1042C000BE043E13CDCF03C00FEF17E0CFCF00EEFB
:1042D00017E0CCCF2093BF041092C004CDCFB8011B
:1042E000D8CF24E632E04AE852E560EE77E082E09B
:1042F0000E94C52CD1CFD0931F02C0931E0280E034
:1043000090E0CDB7DEB7E6E00C94483580911E0210
:1043100090911F028431910538F0449790931F02C9
:1043200080931E020E94A22080E090E008951092E7
:104330001F0210921E020E94A22080E090E00895C9
:1043400080911C0290911D0201976AE070E00E942A
:1043500080342AE0269FC001279F900D112490935E
:104360001F0280931E020E94A22080E090E0089528
:10437000A5E0B0E0EEEBF1E20C94203580E090E0B7
:104380000E94DA29198204E110E024E130E03D8343
:104390002C838C809D803AE0830E911CAC80BD8084
:1043A0008AE0A81AB1082FEF3FEFA801B401C501B8
:1043B0000E949F2A68019AE0C90ED11C78012AE068
:1043C000E21AF1082FEF3FEFA601B7018C819D8122
:1043D0000E94952A0E941C2E8111FCCF0E941C2E47
:1043E0008823E1F30E94882F60931B0670931C06BC
:1043F00080931D0690931E0620EE37E0A801B401BD
:10440000C5010E949F2A20EE37E0A601B7018C81EA
:104410009D810E94952A60911B0670911C068091D7
:104420001D0690911E0639813230D1F0333019F1DA
:10443000313051F03B011C0180913B0190913C01D6
:1044400044979D838C8324C02B01280E391E3694FB
:10445000279400913D0110913E010451110918C0AB
:10446000460E571E569447949B838A8324E130E07E
:104470003D832C830DC0660E771E769467942A8147
:104480003B81820F931F9C01369527953B832A839E
:104490003FEF89E698E1315080409040E1F700C05D
:1044A000000029812F5F2983243009F072CF0E94F8
:1044B0001C2E8111FCCF60913B0170913C0180E08A
:1044C00090E00E946C366B017C01C201861997094D
:1044D0009D838C83BC01990F880B990B0E946E36CB
:1044E0004B015C0120E030E040E252E4C701B6013C
:1044F0000E9457359B01AC01C501B4010E94C4352F
:10450000A70196010E94FA360E9436362C813D8121
:10451000621B730B77FF02C06F5F7F4F75956795C6
:10452000661A770A460E571E60913D0170913E0152
:1045300080E090E00E946C366B017C018A819B8157
:10454000821993099D838C83BC01990F880B990B69
:104550000E946E364B015C0120E030E040E252E404
:10456000C701B6010E9457359B01AC01C501B401DA
:104570000E94C435A70196010E94FA360E94363681
:104580002C813D81621B730B77FF02C06F5F7F4FF1
:1045900075956795261A370A8A819B81860F971F22
:1045A0009B838A839F938F933F922F925F924F9228
:1045B0007F926F9285E492E09F938F9384EB94E0D7
:1045C0009F938F930E94E13760913D0170913E016E
:1045D0007695679524EBE22E24E0F22E00E010E0C1
:1045E0002FEF3FEF41E084E190E00E94752C0FB681
:1045F000F894DEBF0FBECDBF0E941C2E8823E1F3CE
:10460000B3018DEB91E00E94FA3DB20189EB91E09C
:104610000E94FA3DB1018BEB91E00E94FA3D6A8164
:104620007B8187EB91E00E94FA3D80E090E0259647
:10463000E2E10C943C35A7E1B0E0E1E2F3E20C9456
:1046400020351D8A80912102E0914001F0914101C5
:1046500095E0899FE00DF11D112484819D899817B3
:1046600008F082C0228133819D8984E1989FA00156
:104670001124DE01119680E090E0FA01E80FF91FA5
:10468000E20FF31FE491ED93019684319105A9F7B0
:10469000E989FA89E080E1FE63C0E2FE08C0EFE14B
:1046A000F0E0FC87EB8780EE9FEF988B8F874B8441
:1046B0005C848D809E80E985FA85FF8BEE8B6B8014
:1046C0007C802F803884260C371CAD84BE84E0FAB1
:1046D000EE24E0F89F01280D391D620101E0A101DF
:1046E000B401C3010E94AB2AC980DA802F853889C2
:1046F000C40106976E897F8976956795680F791F43
:104700007601820142E0C3010A960E94752CF601EF
:104710008081843429F58181803311F12401F8E10D
:104720004F0E511C310182E0681A710898E0890E21
:10473000911CE2E12E1A310805E115E09201A30176
:10474000B401C1010E94152DF60183818C3341F41F
:1047500000E018EF9201A301B401C1010E94442AB4
:10476000FD89FF5FFD8B6ECF6796E2E10C943C35CF
:104770004096FC01A591B4918C9182FB992790F908
:10478000909590FB82F98C938091B70582FB9927D5
:1047900090F9909590FB82F98093B7050E941B23B6
:1047A00080E090E008954096FC01A591B4918C9131
:1047B00082FF08C08091B70581608093B7058C9116
:1047C0008B7F09C08091B70580FF08C08E7F8093E2
:1047D000B7058C9184608C930E941B2380E090E04D
:1047E00008954096FC01A591B4918C9182FB992784
:1047F00090F9909590FB82F98C930E941B2380E0A6
:1048000090E00895AF92BF92CF92DF92EF920F9314
:10481000CF93DF93CBE3D1E0488159814B505109CD
:10482000A12CB12C8AE8C82E82E5D82EE12C01E01B
:1048300028E131E068E270E08AE090E00E94AB2A73
:10484000488159814B50510999E5C92E9EECD92ECA
:1048500000E028E131E068E270E08AE090E00E9448
:10486000AB2A488159814C50510927E131E069E276
:1048700070E08BE090E00E94AB2A0E941B238FEF38
:104880009FEF9093500180934F010E94A220DF91EF
:10489000CF910F91EF90DF90CF90BF90AF900895A0
:1048A000AF92BF92CF92DF92EF920F93CF9340914E
:1048B0003B0150913C014B505109A12CB12C8AE88D
:1048C000C82E82E5D82EE12C01E028E131E068E233
:1048D00070E08AE090E00E94AB2A40913B01509149
:1048E0003C014B50510999E5C92E9EECD92E00E0B0
:1048F00028E131E068E270E08AE090E00E94AB2AB3
:1049000040913B0150913C014C50510927E131E06D
:1049100069E270E08BE090E00E94AB2A6091400178
:104920007091410140E050E020E030E080912102B0
:10493000FB0195E0899FE00DF11D1124848190E039
:1049400002972817390750F50280F381E02DE40F14
:10495000F51F7096A591B491E0913F01F0E0022E11
:1049600002C0F595E7950A94E2F78C91E0FB82F995
:104970008C9390912102FB01C5E09C9FE00DF11DFD
:104980001124E481F0E033972E173F0711F48B7F59
:104990008C932F5F3F4F4C5E5F4FC8CF0E941B230D
:1049A000CF910F91EF90DF90CF90BF90AF9008958F
:1049B000A0E0B0E0EEEDF4E20C942835CBE3D1E0DA
:1049C0004881598146505109A12CB12C8AE8C82E42
:1049D00082E5D82EE12C01E025EF30E064E670E0BE
:1049E00085E090E00E94AB2A4881598146505109E8
:1049F00099E5C92E9EECD92E00E025EF30E064E663
:104A000070E085E090E00E94AB2A488159814750D0
:104A1000510924EF30E065E670E086E090E00E9406
:104A2000AB2A2CE3E22E22E0F22E0AE812E528E07F
:104A30003CEF42E069E670E086E490E00E94502C92
:104A4000688179816850710928E03CEF4AE750E0BD
:104A500087E090E00E949F2A0E941B23CDB7DEB71B
:104A6000EAE00C944435A0E0B0E0E9E3F5E20C9410
:104A70002835EC01162F60911F0670912006809159
:104A80003D0190913E0140978617970718F481E009
:104A9000809323069B01295F3F4F40913B0150913A
:104AA0003C014B505109A12CB12C8BE7C82E85E25B
:104AB000D82EE12C01E080912106909122060E94DF
:104AC000AB2A60911F06709120068091210690917B
:104AD00022067E01112341F00BE715E22FEF3FEF95
:104AE00041E00E94502C07C00BE715E22FEF3FEF8B
:104AF00041E00E94752C80911F0690912006089637
:104B00009093200680931F06209123062223E1F034
:104B100020913D0130913E01285031092817390775
:104B200068F480912102843019F48AE090E002C098
:104B30008CE191E09093200680931F0680911F06E0
:104B4000909120060E94C829CDB7DEB7EAE00C9408
:104B5000443561E00E9433250895A0E0B0E0E3EB26
:104B6000F5E20C94283584E190E09093220680933E
:104B700021068CE191E09093200680931F060E940D
:104B80002A2944E050E060E270E080911F06909195
:104B900020060E948E2980911F06909120060E9477
:104BA000C8290E94232980E090E00E94DA298EE043
:104BB000E82E82E0F82E00E010E028E03CEF42E032
:104BC0006AE070E084E190E00E94502C92E0E92ECF
:104BD00092E0F92E28E03CEF41E062E170E080EAEB
:104BE00090E00E94502CCBE3D1E06881798128E0ED
:104BF0003CEF4EE150E080E090E00E949F2A0E944E
:104C00001B232A813B8121503109488159814B5016
:104C10005109A12CB12C6BE7C62E65E2D62EE12CF2
:104C200001E068E171E08AE090E00E94AB2A109216
:104C3000230660911F0670912006809121069091B5
:104C400022060E94BC2C8FE095E00E94A92570E806
:104C5000E72E0BE715E22FEF3FEF41E064E271E052
:104C600084E190E00E94D12BCDB7DEB7EAE00C944E
:104C70004435EF920F931F938BE795E20E94DA2958
:104C80008AE090E09093220680932106909320067C
:104C900080931F0646E050E060E371E00E948E2999
:104CA00080911F06909120060E94C8291092230629
:104CB00060911F0670912006809121069091220636
:104CC0000E94BC2C8FE095E00E94A92580E8E82E88
:104CD0000BE715E22FEF3FEF41E062E170E08AE081
:104CE00090E00E94D12B81E080930F0284E08093BA
:104CF000210280E090E01F910F91EF90089560E015
:104D00000E9433250895A2E2B0E0E9E8F6E20C94AF
:104D10002D358C01F62E82E28F1588F442E250E0A8
:104D2000B801CE0101960E94D23760E0CE01019613
:104D30000E9433258EEDF80E0E5D1F4FECCF60E024
:104D4000C8010E943325A296E5E00C944935A0E005
:104D5000B0E0EDEAF6E20C942A3580911D069091C0
:104D60001E068D9768E170E00E948034C0911E029B
:104D7000D0911F022A97C60FD71F61E0CE010E9473
:104D800095188091B80584FF67C0E091BE05F09149
:104D9000BF05C080D180E280F380C482D582E682E4
:104DA000F7828091B4048E3209F03FC08091B5043F
:104DB0008E32D9F5C114D104E104F10439F48FE243
:104DC00090E0909343018093420137C060E080E01F
:104DD00090E00E949518E091BE05F091BF0580819A
:104DE0009181A281B38184839583A683B78300E0F8
:104DF00010E061E0C8010E949518E091BE05F091B5
:104E0000BF0580819181A281B381C816D906EA06C7
:104E1000FB0629F4C482D582E682F78206C00F5FC2
:104E20001F4F0F3F110529F7F5CF4CE050E064EB21
:104E300074E082E491E00E94D23710921F02109237
:104E40001E0210921D0210921C028FEF9FEF909392
:104E5000500180934F011CC0E4EBF4E0019000206E
:104E6000E9F73197BF01645B74406093240684EBDB
:104E700094E00E948326D0935001C0934F0180910B
:104E80001E0290911F020A9790931F0280931E02A8
:104E90000E94A22061E0CE010E94951880E090E07F
:104EA000CDB7DEB7E8E00C944635EF92FF920F9352
:104EB0001F93CF930E949F2DC82F0E9401298EEA35
:104EC00091E00E94C83D80933F0181700E94392982
:104ED0000E9431299F938F938EE292E09F938F934C
:104EE00084EB94E09F938F930E94E13784EBE82E4C
:104EF00084E0F82E00E010E02FEF3FEF42E062E2A6
:104F000071E084E190E00E94752C0F900F900F905B
:104F10000F900F900F90CC2379F08DEB91E00E94D1
:104F2000D63D019629F40E9423290E94B82104C08D
:104F30000E941C2E8111F7CFCF911F910F91FF90EE
:104F4000EF900895FF920F931F93CF93DF93F0900C
:104F50003F01F0FAFF24F0F810923F018091210206
:104F6000A0914001B091410175E0879FA00DB11D56
:104F7000112460E0262F30E014968C91149790E075
:104F8000FC0132972E173F0714F51296ED91FC9114
:104F9000139774E1679FE00DF11D11247096059140
:104FA0001491E8010397281739077CF4888182FB64
:104FB000442740F950E0CA0101C0880F2A95EAF75A
:104FC00090913F01892B80933F016F5FD3CF609118
:104FD0003F018EEA91E00E94DC3D888182FD0EC097
:104FE00080913F018170F81661F16FEF7FEF8DEBDB
:104FF00091E00E94FA3D0E94552723C0CCE3D2E005
:1050000006E911E08EA580FF0EC04C8D5D8D6E8D82
:105010007F8DC8010E94EE3D68A579A5C801049660
:105020000E94FA3D06C04FEF5FEFBA01C8010E942F
:10503000EE3D68960A5F1F4F82E0CC39D80711F722
:10504000CFCF0E941A2080E090E0CDB7DEB7E5E038
:105050000C944935A0E0B0E0E0E3F8E20C94283588
:105060000E940E2F362F272F60931B0670931C066D
:1050700080931D0690931E0680912102A09140010D
:10508000B091410195E0899FA00DB11D11241496A6
:10509000AC901497832F922F00911D0610911E063D
:1050A00040E050E0B12CBA1451F112962D913C9190
:1050B0001397240F351FF9013296C590D490F9014A
:1050C0003496E590F490F9013696C591D491F901A2
:1050D000389665917491C816D90668F4CC0DDD1D1B
:1050E0008C179D0740F4E016F10628F46E0D7F1D25
:1050F0000617170738F0B3944C5E5F4FD4CF80E0AB
:1051000090E001C0C901CDB7DEB7EAE00C944435A8
:1051100084B1836084B98AB18C6F8AB987B18F6199
:1051200087B988B18B6088B98FE39CE90197F1F763
:1051300000C00000089544988FE59AEE0197F1F7BA
:1051400000C00000449A8FE59AEE0197F1F700C085
:10515000000008959BB19370282F2C7F922B9BB950
:1051600095B19C7F8370892B85B94198419A0895A8
:1051700040982FEF89EF90E0215080409040E1F778
:1051800000C0000029B193B1409A2C7F892F837011
:10519000822B0895429843980E94AA28439A089522
:1051A000CF93C82F429A4398892F0E94AA288C2F08
:1051B0000E94AA28439ACF910895CF9384B18C7FFF
:1051C00084B98AB183708AB9429A43980E94B828F8
:1051D000C82F0E94B828439A94B1936094B99AB1A9
:1051E0009C6F9AB92C2F30E0322F2227A901482B2F
:1051F000CA01CF910895429A43980E94AA28439ADF
:105200000895CF93DF930E9488280E949B282FEF58
:105210008DEE92E0215080409040E1F700C0000008
:10522000C6E1D7E0FE0184910E94CA28FE013196B2
:1052300084910E94FB282296F7E0C032DF0791F7A5
:10524000DF91CF91089588E20E94CA288CE30E94E2
:10525000FB28089588E20E94CA2880E00E94FB286B
:10526000089580E00E94CA280E94DD280E94DD285F
:105270000895CF93C82F86E10E94CA28CC2321F03D
:10528000C13029F488E901C088E40E94FB28CF914D
:105290000895A0E0B0E0EFE4F9E20C942A35D82EAE
:1052A000C92E162F072FF42EE52EE90182E00E9469
:1052B000CA288C2D0E94FB2883E00E94CA288D2DCD
:1052C0000E94FB2884E00E94CA288E2D0E94FB28A1
:1052D00085E00E94CA288F2D0E94FB2886E00E944C
:1052E000CA28802F0E94FB2887E00E94CA28812FAD
:1052F0000E94FB2888E00E94CA288D2F0E94FB286C
:1053000089E00E94CA288C2F0E94FB2882E20E941A
:10531000CA28CDB7DEB7E8E00C944635EF92FF928D
:105320000F931F93CF93DF93F82EE92E162F072F9D
:10533000EA018EE00E94CA288E2D0E94FB288FE091
:105340000E94CA288F2D0E94FB2880E10E94CA2853
:10535000802F0E94FB2881E10E94CA28812F0E9491
:10536000FB2882E10E94CA288D2F0E94FB2883E13E
:105370000E94CA288C2F0E94FB2881E00E94CA2824
:1053800088E00E94FB28CDB7DEB7E6E00C944835F4
:10539000CF93DF93EC0184E10E94CA288D2F0E94F5
:1053A000FB2885E10E94CA288C2F0E94FB28DF91F0
:1053B000CF910895CF92DF92EF92FF92CF93DF9338
:1053C000EC0120915101309152012150310940915D
:1053D0005301509154014150510960E070E080E068
:1053E00090E00E944929C12C8CE2D82EEE24E3944F
:1053F000F12CCE010E94D02881E0C81AD108E10822
:10540000F108B9F7DF91CF91FF90EF90DF90CF9047
:105410000895CF92DF92EF92FF920F931F93DA01DC
:10542000A81BB90B1196F901E61BF70B3196AE9F3D
:105430006001AF9FD00CBE9FD00C1124E12CF12C49
:105440000E944929C114D104E104F10449F0C801C2
:105450000E94D02881E0C81AD108E108F108F2CFF3
:105460001F910F91FF90EF90DF90CF900895CF9311
:10547000DF93EA019B01AC010E944929CE010E9401
:10548000D028DF91CF910895A0E0B0E0EAE4FAE2FD
:105490000C9422357C01EB013A0129016A01C81AFA
:1054A000D90A5901A61AB70ACC0CDD1CAA0CBB1CE0
:1054B000A8010E94372AAC14BD04C8F4C601969511
:1054C00087954501881A990AE614F70449F197FC73
:1054D00003C021968C189D088FEFE81AF80A8A0CF1
:1054E0009B1CA801BE01C7010E94372AEDCFC50150
:1054F000969587954601881A990AC415D50581F0B5
:1055000097FC05C08FEFE81AF80A8A189B082196C5
:105510008C0C9D1CA801BE01C7010E94372AEDCF4B
:10552000CDB7DEB7E0E10C943E350F931F938901B0
:105530009A01AC010E94092A1F910F9108950F93BF
:105540001F93FB01BA0189019A01AF010E94092A48
:105550001F910F9108954F925F926F927F928F9259
:105560009F92AF92BF92CF92DF92EF920F931F93D1
:10557000CF93DF933C014B01EA012901013021F473
:1055800086010E94092A16C09601A2010E94952A4E
:105590009601A201B401CE010E94952A9601A401B0
:1055A000BE01C3010E949F2A9601A201BE01C30150
:1055B0000E949F2AEE20A1F0A501B401C3010E9420
:1055C000372AA501B201C3010E94372AA501B401FF
:1055D000CE010E94372AA501B201CE010E94372ACE
:1055E000DF91CF911F910F91EF90DF90CF90BF90FF
:1055F000AF909F908F907F906F905F904F900895A5
:10560000ADE0B0E0E6E0FBE20C9420357C013B012C
:105610005D874C872B8781E090E09C01241B350B34
:105620003A83298317014B017C836B83270143E075
:1056300050E058874F839E838D832D813E8121507A
:1056400031093A872987CC84DD84C60CD71C3B8579
:10565000313039F59801A601B101C2010E949F2A9B
:105660009801A3018C859D85481B590BB101C2018E
:105670000E949F2A98014B815C81AC84BD84AE0C52
:10568000BF1CB50167018C859D85C81AD90AC60162
:105690000E949F2A9801A401B501C6010E949F2A79
:1056A00038C0A801B601C1010E94372AA8016B8148
:1056B0007C81AC84BD84AE0CBF1CC5010E94372A1E
:1056C000A801B601C2010E94372AA8016B817C8122
:1056D00067012C853D85C21AD30AC6010E94372A6C
:1056E000A801B401C5010E94372AA80153018C8585
:1056F0009D85A81AB90AB501C1010E94372AA801DF
:10570000B501C2010E94372AA801B401C6010E9456
:10571000372A29813A8137FF0BC02D813E8149818B
:105720005A818F819885480F591F5A83498316C023
:105730002D813E8189859A854C855D85841B950BDD
:10574000880F991F059649815A81480F591F5A831E
:1057500049838C859D8501979D878C874D815E81CE
:105760004F5F5F4F5E834D838F8198850296988748
:105770008F8391E0491A51084FEF241A340A8B8124
:105780009C8101969C838B8391E0891A91084C85BA
:105790005D85421753070CF050CF2D96E2E10C9433
:1057A0003C352F923F924F925F927F928F929F92C1
:1057B000AF92BF92CF92DF92EF92FF920F931F931F
:1057C000CF93DF93FC01542E4901411102C05524AF
:1057D0005394852D90E09C018E179F0708F4CF010C
:1057E00043E0220F331F4A95E1F7AB0141505109C5
:1057F000240F351FAC0141505109E5E05E9E400D7C
:10580000511D11240E94492985E0E89E7001112450
:10581000C12CD12CE0EAEE1AF10822242394312C79
:105820000C2C02C0220C331C0A94E2F7712CA12C20
:10583000B12CF701EA0DFB1DE05EF84FC491D0E0FA
:10584000C221D321412C209711F0C40101C0C8010D
:105850000E94D02843945410F6CF8FEFA81AB80AAC
:10586000E5E0AE16B10429F773945710E0CF8FEF3F
:10587000C81AD80AE8E0CE16D10479F6DF91CF91A4
:105880001F910F91FF90EF90DF90CF90BF90AF905E
:105890009F908F907F905F904F903F902F900895B2
:1058A000A0E0B0E0E6E5FCE20C9421356C015B0180
:1058B000342E4901380186E0489F20011124F70168
:1058C000E490EF012196EE2059F083019401432DDD
:1058D000B501C6010E94D12BC40CD51CFE01F0CF2E
:1058E000CDB7DEB7E1E10C943D35A0E0B0E0EBE7E9
:1058F000FCE20C9421353C016B01342E5901480126
:1059000086E0489F20011124E701E9908401950178
:10591000432DB601C3010E94D12B640C751C8881F4
:105920008052803690F3CDB7DEB7E1E10C943D357F
:10593000A0E0B0E0EEE9FCE20C942035EC015B0164
:10594000D42E4901380186E0489F10011124270117
:10595000F201E1902F01830194014D2DB501CE019B
:105960000E94D12BC20DD31DCA94C110F1CFCDB767
:10597000DEB7E2E10C943C3590932806809327062D
:1059800070932606609325060895EF92FF920F9379
:105990001F93CF93C82F80912506909126067901F9
:1059A0008A019B014C2FBC0180912706909128060B
:1059B0000E94502C80912506909126062CE0C29FD3
:1059C000800D911D11249093260680932506CF917A
:1059D0001F910F91FF90EF900895EF92FF920F9318
:1059E0001F93CF93C82F80912506909126067901A9
:1059F0008A019B014C2FBC018091270690912806BB
:105A00000E94752C80912506909126062CE0C29F5D
:105A1000800D911D11249093260680932506CF9129
:105A20001F910F91FF90EF900895A0E0B0E0EBE19F
:105A3000FDE20C942635FC01EB015901261B370BC6
:105A4000DA01A81BB90B0E94EF346B017C019501B0
:105A50002150310941505109BE01CF010E9449290D
:105A6000E801812C912C54018C149D04AE04BF04D8
:105A700061F0FE01859194910E94D0288FEF881AE1
:105A8000980AA80AB80A2296EFCFCDB7DEB7ECE0A5
:105A90000C944235E0912E06F0912F0681E090E0C3
:105AA0009C0100902B0602C0220F331F0A94E2F7DC
:105AB000322F3095418134233183E0912E06F091CD
:105AC0002F063281232B228338B1AC01009030069F
:105AD00002C0440F551F0A94E2F7242F2095232378
:105AE00028B937B1AC010090290602C0440F551FF8
:105AF0000A94E2F7242F2095232327B938B1AC016B
:105B00000090290602C0440F551F0A94E2F7242F83
:105B10002095232328B9E0912C06F0912D060090C2
:105B20002A0602C0880F991F0A94E2F78095928195
:105B30008923828385E38A95F1F70000089587E839
:105B400080937A0086EB91E00E94C83D8F3F31F14F
:105B50008093290685EB91E00E94C83D80932B0637
:105B600082EB91E00E94C83D80932A068FEA91E083
:105B70000E94C83D8093300683EB91E00E94D63DA1
:105B800090932F0680932E0680EB91E00E94D63DE5
:105B900090932D0680932C0681E0089580E008956F
:105BA00048B181E090E09C010090290602C0220FDC
:105BB000331F0A94E2F7242B28B948B19C010090C6
:105BC000300602C0220F331F0A94E2F7242B28B9B3
:105BD000E0912E06F0912F069C0100902B0602C04A
:105BE000220F331F0A94E2F73181232B218347B11F
:105BF0009C010090300602C0220F331F0A94E2F786
:105C0000242B27B947B19C010090290602C0220F1E
:105C1000331F0A94E2F7242B27B9E0912C06F09168
:105C20002D0600902A0602C0880F991F0A94E2F7F9
:105C30009181892B81830895CF93DF93F8940E94FB
:105C40004A2DE0912E06F0912F06C081D0E0009001
:105C50002B0602C0D595C7950A94E2F7C170DD27DF
:105C600081E0C8270E94D02D78948C2FDF91CF91AE
:105C70000895E0912E06F0912F0620912B06409179
:105C80003006882309F45BC081E090E0BC0102C0CB
:105C9000660F771F2A95E2F79B0120953181322309
:105CA0003183E0912E06F0912F0632812323228347
:105CB00057B19C0101C0220F4A95EAF7252B27B95D
:105CC00038B1AC010090300602C0440F551F0A9451
:105CD000E2F7242F2095232328B937B1AC01009097
:105CE000290602C0440F551F0A94E2F7242F20957D
:105CF000232327B938B1AC010090290602C0440F14
:105D0000551F0A94E2F7242F2095232328B9E09108
:105D10002C06F0912D0600902A0602C0880F991FCC
:105D20000A94E2F79181982B9183E0912C06F091EF
:105D30002D069281892B8283809129065AC081E0A9
:105D400090E0BC0102C0660F771F2A95E2F79B0125
:105D50003181322B3183E0912E06F0912F06209570
:105D600032812323228337B1BC0102C0660F771F23
:105D70004A95E2F7262F2095232327B938B1AC01A5
:105D80000090300602C0440F551F0A94E2F7242FFA
:105D90002095232328B947B19C010090290602C011
:105DA000220F331F0A94E2F7242B27B948B19C0134
:105DB0000090290602C0220F331F0A94E2F7242B19
:105DC00028B9E0912C06F0912D0600902A0602C019
:105DD000880F991F0A94E2F7809591819823918307
:105DE000E0912C06F0912D06928189238283809187
:105DF0003006806480937C0072E07A95F1F700C0F1
:105E000080917A00806480937A0080917A0086FD88
:105E1000FCCF80917800909179000895A8E0B0E0DF
:105E2000E4E1FFE20C942035F89440905301509047
:105E30005401612C712C89EB91E00E94D63D8C01BC
:105E40008DEB91E00E94D63D6C01E12CF12C80E0BD
:105E50000E94392E98878F83809051019090520133
:105E6000940140E050E029833A834B835C8387EBC5
:105E700091E00E94D63D9E838D838BEB91E00E9442
:105E8000D63D4C01A12CB12C81E00E94392E1C0181
:105E90000E94D02D78944F815885CA01A0E0B0E0CF
:105EA0009C01AD012C193D094E095F09C301B201E6
:105EB0000E94643420E030E0A90198012C193D09CA
:105EC0004E095F090E94CA346901C101A0E0B0E037
:105ED0009C01AD01281939094A095B0969817A8158
:105EE0008B819C810E946434AD81BE818D0120E054
:105EF00030E0A9019801281939094A095B090E9473
:105F0000CA347901C701B6012896E2E10C943C3508
:105F10000F931F93CF93DF93F89480E00E94392E64
:105F20008C0181E00E94392EEC010E94D02D7894E2
:105F3000B801CE01DF91CF911F910F910895CF92BB
:105F4000DF92EF92FF92CF93DF9320E330E040E0C7
:105F500050E0BA0180E00E949D1A8091B40481341F
:105F600009F05EC08091B504843509F059C0809174
:105F7000B604883309F054C08091B704883509F01D
:105F80004FC08091B8049091B904019709F048C0BE
:105F90008091BA049091BB04019709F041C08091AF
:105FA000C604813011F092E101C09AE19093350668
:105FB000823019F080E890E002C080E091E0909398
:105FC000340680933306C090D004D090D104E09082
:105FD000D204F090D304C7E3D6E020E230E0B7016A
:105FE000A60180E00E949D1A892B29F48091330636
:105FF0009091340617C0C992D992E992F992809192
:10600000B4049091B504A091B604B091B704C80E41
:10601000D91EEA1EFB1E86E0CF3DD807F1F6E6CF7B
:1060200080E090E0DF91CF91FF90EF90DF90CF90F4
:106030000895A0E1B0E0EFE1F0E30C942035FB011E
:10604000588B4F87019798878F8380913506282F2B
:1060500030E03A8729878F819885B9010E94803482
:1060600001E0060F80E1AF85B8898C9380913306FB
:1060700090913406918380830E944B32EFE4F2E3E7
:106080003197F1F700C0000080913606081761F1E2
:10609000E02EE81AE7FCE194C12CD12C0E2C000C68
:1060A000FF08CE14DF0498F40E944B32882329F0B5
:1060B00087EE91EC0197F1F704C0AFECB2E51197D0
:1060C000F1F700C00000BFEFCB1ADB0AEACF0E9455
:1060D0004B32882349F0EFEFF3EF21E0E150F0403D
:1060E0002040E1F700C00000009336060E944432D1
:1060F0006C0110E001501109A801440F551F440F15
:10610000551F5E834D83FA01E95CF94F80809180D1
:10611000A280B38081149104A104B10419F4E12C8C
:10612000F12C92C120E230E0B501A40180E00E9490
:106130009D1A8091BC0490E00817190781F7209000
:10614000BE043090BF042114310449F38091C80487
:106150009091C904A091CA04B091CB04880E991EF5
:10616000AA1EBB1E28E030E0B501A40180E00E9419
:106170009D1A8091B4049091B504A091B604B09199
:10618000B704880E991EAA1EBB1EC10123E0880F0A
:10619000991F2A95E1F7A5019401281B390B4109A4
:1061A00051092B873C874D875E8734E03C8300E0B4
:1061B00010E01B82812C912C5401E12CF12C4B849A
:1061C0005C846D847E841A82198228E030E0B301F9
:1061D000A20180E00E949D1A892B09F44EC02091F3
:1061E000B50424FD45C08F81988569857A850E9414
:1061F00080348F5F9091B40489133AC08091B604C3
:106200009091B704AC014C195D090115110571F0AD
:10621000141615061CF417FD09C005C041155105DB
:1062200039F117FF25C04017510714F59093320636
:106230008093310622FD04C0AF85B8892C9305C038
:10624000822F8260EF85F8898083AF85B8898C9131
:1062500086FF03C0BB81BF5FBB838090B804909072
:10626000B904A090BA04B090BB048A01E980FA8016
:10627000E8E04E0E511C611C711C29813A812F5F90
:106280003F4F3A8329832216330609F09ECFAF850C
:10629000B8898C91811114C0809131069091320699
:1062A0009093B5058093B405EF85F88980818F7749
:1062B00089838083FB81F11115C00FEF1FEF54C05C
:1062C0000E9444329C0186549A498B3B45E69407D0
:1062D00008F0C9010E942E325C8151505C8351113B
:1062E0006ECFDACFED81FE81E95CF94F40805180BD
:1062F000628073808091C8049091C904A091CA04FF
:10630000B091CB04480E591E6A1E7B1E0FEF1FEF83
:1063100028E030E0B301A20180E00E949D1A409184
:10632000B4045091B5046091B6047091B70441155E
:1063300051056105710599F08091B90490E0E81666
:10634000F90641F48091B804803121F40091BA0437
:106350001091BB04440E551E661E771ED9CFAF8523
:10636000B8898C918F7B8C9381149104A104B10422
:10637000A1F02091330630913406ED81FE81E95C75
:10638000F94F4081518162817381480D591D6A1D09
:106390007B1D80E00E949D1A7C018981882311F079
:1063A000E12CF12C17FF0AC0809131069091320642
:1063B000C816D906E0F086549A4919C0D801AC54E1
:1063C000BB4F5D0100E011E02091330630913406AF
:1063D000C501845B94408217930730F70E94B3375E
:1063E000B8010E949434F50181935F01EDCF9C01C7
:1063F0002C193D098AEB95E6B1010E948034C20E4A
:10640000D31EFBEBCF16F5E6DF0620F02AEBC21A0F
:1064100025E6D20ACB018C0D9D1D8B3B35E69307FB
:1064200010F08A5B95460E942E320E944B328823E0
:1064300029F08FE39FE10197F1F704C0AFE3BFE1DB
:106440001197F1F700C00000EF85F88980818095F1
:106450008083C7016096E2E10C943C352091840072
:1064600030918500369527958217930718F4B19AD5
:10647000B19BFECF20918400309185003695279501
:1064800028173907B8F3089580918400909185000A
:1064900096958795089580913F0183FB882780F921
:1064A00008952091E1063091E2063695279540E067
:1064B00050E060E472E48FE090E00E94A834C901EB
:1064C00001970E94181F08958F929F92AF92BF92DA
:1064D000EF92FF920F931F93CF93DF93EC014C0148
:1064E000A12CB12CE091BE05F091BF0542895389E2
:1064F0006489758984169506A606B70608F05CC0FF
:10650000415051096109710997E076956795579552
:1065100047959A95D1F74F5F5F4F6F4F7F4F7F93AE
:106520006F935F934F93CE01880F892F881F990B2C
:10653000919501969F938F9389E399E09F938F9311
:1065400084EB94E09F938F930E94E13734EBE32E2A
:1065500034E0F32E0AE812E520EE3FEF42E064E873
:1065600070E083E290E00E94752C20E830E0B501F5
:10657000A40180E00E949D1AE4E3F5E02DB73EB748
:10658000265F3F4F0FB6F8943EBF0FBE2DBF34E0DD
:10659000E43BF30719F092919383F9CF87FD06C08E
:1065A0009AEF9093B6048093360503C09CEF9093C6
:1065B000B604C80FD11D18C083E3E82E89E0F82E79
:1065C0000AE812E520EE3FEF42E064E870E083E283
:1065D00090E00E94502C83E890E00E949A058EEF94
:1065E0008093B604C0E0D0E085E58093B404809346
:1065F000B50463E870E084EB94E00E94381F63E820
:1066000070E084EB94E00E94091F0E94311F8FEF1D
:1066100095EA2EE0815090402040E1F700C0000054
:10662000CE01DF91CF911F910F91FF90EF90BF901E
:10663000AF909F908F90089528E030E040E050E0C8
:10664000BA0180E00E949D1A9091B4048091B70530
:10665000963471F49091B504953551F49091B60447
:106660009A3431F49091B704993411F4826001C0E6
:106670008D7F8093B7058091B70582FF03C088EEB8
:1066800093E002C088E592E09093E2068093E106F1
:106690000E9451321092E0061092DF060895A0E0A9
:1066A000B0E0E5E5F3E30C9424356C014601A12C40
:1066B000B12CE091BE05F091BF0582899389A48930
:1066C000B58988169906AA06BB0608F045C028E0D9
:1066D00030E0B501A40180E00E949D1AC091B80489
:1066E000D091B9048091B4048436B1F48091B5049A
:1066F000813671F58091B604843751F58091B704E5
:10670000813631F58091DF069091E00601969093F5
:10671000E0068093DF0620C08236D1F48091B50474
:106720008136B1F48091B604853791F48091B70435
:10673000843671F48091B70582FDB8CF8091BA0498
:106740009091BB049093E2068093E1060E9451323F
:106750002896CC0EDD1EAACF84EB94E06090BA049C
:106760007090BB04C091B804D091B9047F926F922D
:10677000DF93CF932091E2062F932091E1062F9390
:1067800023E139E03F932F939F938F930E94E1374A
:1067900094EBE92E94E0F92E0AE812E520EE37E0BA
:1067A00041E069E970E08FE090E00E94752C8DB7C0
:1067B0009EB70A960FB6F8949EBF0FBE8DBFC30159
:1067C000009741F0EFE9FFE03197F1F700C00000DA
:1067D0000197F6CFE091BE05F091BF0582899389BC
:1067E000A489B58988169906AA06BB0608F064C074
:1067F0008091E0068F938091DF068F9385E099E08A
:106800009F938F9384EB94E09F938F930E94E13743
:1068100084EBE82E84E0F82E0AE812E520EE3FEF44
:1068200042E064E870E083E290E00E94752C86010B
:10683000085F1F4F0F900F900F900F900F900F90C9
:10684000DD24D39480E091E0209731F1C130F1E074
:10685000DF0720F05E01BA94EC0102C0A12CB12C3C
:10686000A80160E070E09E0180E00E949D1A080F80
:10687000191FBE0184EB94E00E94381FDD2041F017
:106880008091B6048E3F21F41092E0061092DF064C
:10689000D12CCE01E501D8CF8091DF069091E006A2
:1068A000892B61F48FEF93ECE9E081509040E04058
:1068B000E1F700C0000002C000E010E0C801CDB761
:1068C000DEB7EEE00C944035DB018F939F930E947E
:1068D0000D35BF91AF91A29F800D911DA39F900D8B
:1068E000B29F900D11240895991B79E004C0991F5F
:1068F000961708F0961B881F7A95C9F7809508951A
:10690000AA1BBB1B51E107C0AA1FBB1FA617B707D5
:1069100010F0A61BB70B881F991F5A95A9F78095F1
:106920009095BC01CD01089597FB072E16F40094B5
:1069300007D077FD09D00E94803407FC05D03EF4D3
:10694000909581959F4F0895709561957F4F08951B
:10695000A1E21A2EAA1BBB1BFD010DC0AA1FBB1F63
:10696000EE1FFF1FA217B307E407F50720F0A21BD5
:10697000B30BE40BF50B661F771F881F991F1A9442
:1069800069F760957095809590959B01AC01BD016C
:10699000CF010895052E97FB1EF400940E94E13468
:1069A00057FD07D00E94A83407FC03D04EF40C9486
:1069B000E13450954095309521953F4F4F4F5F4FB3
:1069C000089590958095709561957F4F8F4F9F4F5B
:1069D0000895EE0FFF1F0590F491E02D09940E9499
:1069E000F734332312F48A1B9B0B0C940835A29FB7
:1069F000B001B39FC001A39F700D811D1124911D93
:106A0000B29F700D811D1124911D08950E94F734CD
:106A1000B7FF0895821B930B08950E94F734A59F3A
:106A2000900DB49F900DA49F800D911D1124089589
:106A3000B7FF0C940D350E940D35821B930B089502
:106A40002F923F924F925F926F927F928F929F927E
:106A5000AF92BF92CF92DF92EF92FF920F931F936C
:106A6000CF93DF93CDB7DEB7CA1BDB0B0FB6F8941D
:106A7000DEBF0FBECDBF09942A88398848885F845D
:106A80006E847D848C849B84AA84B984C884DF80CE
:106A9000EE80FD800C811B81AA81B981CE0FD11DB2
:106AA0000FB6F894DEBF0FBECDBFED01089550586C
:106AB000BB27AA270E946F350C94C0360E94B236BD
:106AC00038F00E94B93620F039F49F3F19F426F4CB
:106AD0000C94AF360EF4E095E7FB0C94A936E92F41
:106AE0000E94D13658F3BA176207730784079507D7
:106AF00020F079F4A6F50C94F3360EF4E0950B2E05
:106B0000BA2FA02D0B01B90190010C01CA01A001FF
:106B10001124FF27591B99F0593F50F4503E68F15A
:106B20001A16F040A22F232F342F4427585FF3CF9B
:106B3000469537952795A795F0405395C9F77EF46C
:106B40001F16BA0B620B730B840BBAF09150A1F0B5
:106B5000FF0FBB1F661F771F881FC2F70EC0BA0F3B
:106B6000621F731F841F48F4879577956795B795C3
:106B7000F7959E3F08F0B0CF9395880F08F09927BE
:106B8000EE0F9795879508950E94D8350C94C036DE
:106B90000E94B93658F00E94B23640F029F45F3FA7
:106BA00029F00C94A93651110C94F4360C94AF369C
:106BB0000E94D13668F39923B1F3552391F3951BC5
:106BC000550BBB27AA2762177307840738F09F5F0E
:106BD0005F4F220F331F441FAA1FA9F335D00E2E7B
:106BE0003AF0E0E832D091505040E695001CCAF7E8
:106BF0002BD0FE2F29D0660F771F881FBB1F2617AB
:106C000037074807AB07B0E809F0BB0B802DBF0181
:106C1000FF2793585F4F3AF09E3F510578F00C9450
:106C2000A9360C94F4365F3FE4F3983ED4F386958E
:106C300077956795B795F7959F5FC9F7880F911D71
:106C40009695879597F90895E1E0660F771F881F5D
:106C5000BB1F621773078407BA0720F0621B730B10
:106C6000840BBA0BEE1F88F7E09508950E943D361D
:106C70006894B1110C94F43608950E94D93688F0C6
:106C80009F5798F0B92F9927B751B0F0E1F0660FF0
:106C9000771F881F991F1AF0BA95C9F714C0B13031
:106CA00091F00E94F336B1E008950C94F336672F0B
:106CB000782F8827B85F39F0B93FCCF38695779560
:106CC0006795B395D9F73EF4909580957095619549
:106CD0007F4F8F4F9F4F0895E89409C097FB3EF474
:106CE00090958095709561957F4F8F4F9F4F992319
:106CF000A9F0F92F96E9BB279395F6958795779597
:106D00006795B795F111F8CFFAF4BB0F11F460FF56
:106D10001BC06F5F7F4F8F4F9F4F16C0882311F0AE
:106D200096E911C0772321F09EE8872F762F05C0C2
:106D3000662371F096E8862F70E060E02AF09A955D
:106D4000660F771F881FDAF7880F9695879597F952
:106D5000089597F99F6780E870E060E008959FEFDD
:106D600080EC089500240A941616170618060906E2
:106D7000089500240A9412161306140605060895B1
:106D8000092E0394000C11F4882352F0BB0F40F439
:106D9000BF2B11F460FF04C06F5F7F4F8F4F9F4F79
:106DA000089557FD9058440F551F59F05F3F71F0FB
:106DB0004795880F97FB991F61F09F3F79F0879562
:106DC0000895121613061406551FF2CF4695F1DFEB
:106DD00008C0161617061806991FF1CF869571057B
:106DE000610508940895E894BB2766277727CB01AF
:106DF00097F908950E940D370C94C0360E94B23660
:106E000038F00E94B93620F0952311F00C94A93681
:106E10000C94AF3611240C94F4360E94D13670F3E2
:106E2000959FC1F3950F50E0551F629FF001729F2F
:106E3000BB27F00DB11D639FAA27F00DB11DAA1F3E
:106E4000649F6627B00DA11D661F829F2227B00D8B
:106E5000A11D621F739FB00DA11D621F839FA00D16
:106E6000611D221F749F3327A00D611D231F849F66
:106E7000600D211D822F762F6A2F11249F575040BD
:106E80009AF0F1F088234AF0EE0FFF1FBB1F661F38
:106E9000771F881F91505040A9F79E3F510580F001
:106EA0000C94A9360C94F4365F3FE4F3983ED4F387
:106EB000869577956795B795F795E7959F5FC1F7A5
:106EC000FE2B880F911D9695879597F908958F92BF
:106ED0009F92AF92BF92CF92DF92EF92FF92CF93A9
:106EE000DF93EC01688179818A819B81611571054D
:106EF0008105910521F464E279ED8BE597E02DE1C0
:106F000033EF41E050E00E94CA3449015A019B012D
:106F1000AC01A7EAB1E40E940D356B017C01ACEE37
:106F2000B4EFA50194010E941B35DC01CB018C0D4F
:106F30009D1DAE1DBF1DB7FF03C00197A109B0483D
:106F400088839983AA83BB839F77DF91CF91FF903A
:106F5000EF90DF90CF90BF90AF909F908F9008956B
:106F60000E946737089585E591E00E94673708958C
:106F7000A0E0B0E08093550190935601A093570193
:106F8000B09358010895FB01DC014150504048F096
:106F900005900D920020C9F701C01D92415050404C
:106FA000E0F70895FB01DC014150504048F00190AA
:106FB0000D920020C9F701C01D9241505040E0F7EA
:106FC0000895AEE0B0E0E7EEF7E30C942E350D89BE
:106FD0001E898EE08C831A8309838FEF9FE79E833F
:106FE0008D83AE01475E5F4F6F89788DCE0101962C
:106FF0000E941C38EF81F885E00FF11F10822E9659
:10700000E4E00C944A35AEE0B0E0E9E0F8E30C943B
:1070100030358DE08C838B899C899A838983AE017E
:10702000495E5F4F6D897E89CE0101960E94993B32
:107030002E96E2E00C944C35ABE0B0E0E2E2F8E3EF
:107040000C9420356C017B018A01FC0117821682A9
:10705000838181FFCCC1CE0101963C01F601938171
:10706000F70193FD859193FF81917F01882309F4B6
:10707000BAC1853239F493FD859193FF81917F01E7
:10708000853229F4B60190E00E94123DE7CF912CA1
:10709000212C312CFFE1F315D8F08B3279F038F444
:1070A000803279F08332A1F4232D20611DC08D320E
:1070B00061F0803369F4232D216016C0832D826036
:1070C000382EE32DE4603E2E2AC0F32DF8601DC05B
:1070D00037FC2DC020ED280F2A3040F08E32B9F455
:1070E00036FC81C1232D2064322E19C036FE06C025
:1070F0008AE0989E200D1124922E11C0EAE02E9E67
:10710000200D1124222EF32DF0623F2E08C08C3664
:1071100021F4832D8068382E02C0883641F4F701AF
:1071200093FD859193FF81917F018111B3CF982FBA
:107130009F7D9554933028F40C5F1F4F9FE39983F4
:107140000DC0833631F0833771F0833509F059C0B3
:1071500021C0F801808189830E5F1F4F88248394AA
:10716000912C530113C02801F2E04F0E511CF8017D
:10717000A080B18036FE03C0692D70E002C06FEFC1
:107180007FEFC5010E94C93C4C018201F32DFF77BE
:107190003F2E16C0280122E0420E511CF801A080AB
:1071A000B18036FE03C0692D70E002C06FEF7FEF43
:1071B000C5010E94BE3C4C01F32DF0683F2E8201B8
:1071C00033FC1BC0822D90E088169906B0F4B601FE
:1071D00080E290E00E94123D2A94F4CFF50137FC42
:1071E000859137FE81915F01B60190E00E94123DCA
:1071F00021102A9421E0821A91088114910471F7D8
:10720000E8C0843611F0893641F5F80137FE07C031
:1072100060817181828193810C5F1F4F08C0608102
:107220007181072E000C880B990B0E5F1F4FF32DF9
:10723000FF763F2E97FF09C09095809570956195D8
:107240007F4F8F4F9F4FF0683F2E2AE030E0A30121
:107250000E94673D882E861845C0853731F4232D5E
:107260002F7EB22E2AE030E025C0932D997FB92ED3
:107270008F36C1F018F4883579F0B5C0803719F031
:10728000883721F0B0C0E92FE061BE2EB4FE0DC0FA
:10729000FB2DF460BF2E09C034FE0AC0292F2660E2
:1072A000B22E06C028E030E005C020E130E002C088
:1072B00020E132E0F801B7FE07C060817181828170
:1072C00093810C5F1F4F06C06081718180E090E068
:1072D0000E5F1F4FA3010E94673D882E8618FB2D6D
:1072E000FF773F2E36FE0DC0232D2E7FA22E891450
:1072F00058F434FE0BC032FC09C0832D8E7EA82EBC
:1073000005C0B82CA32C03C0B82C01C0B92CA4FE16
:107310000FC0FE01E80DF11D8081803321F49A2D0C
:10732000997EA92E09C0A2FE06C0B394B39404C0EE
:107330008A2D867809F0B394A3FC11C0A0FE06C084
:10734000B21488F4280C922C9B180EC0B21460F46E
:10735000B60180E290E00E94123DB394F7CFB214E0
:1073600018F42B1802C0982C212CA4FE10C0B601D2
:1073700080E390E00E94123DA2FE17C0A1FC03C072
:1073800088E790E002C088E590E0B6010CC08A2D45
:10739000867859F0A1FE02C08BE201C080E2A7FC12
:1073A0008DE2B60190E00E94123D891438F4B601D6
:1073B00080E390E00E94123D9A94F7CF8A94F30103
:1073C000E80DF11D8081B60190E00E94123D811010
:1073D000F5CF222009F442CEB60180E290E00E946F
:1073E000123D2A94F6CFF6018681978102C08FEF75
:1073F0009FEF2B96E2E10C943C3520FD09C0FC0187
:1074000023FD05C022FF02C0738362835183408342
:10741000089544FD17C046FD17C0AB01BC01DA0159
:10742000FB01AA0FBB1FEE1FFF1F1094D1F74A0FDD
:107430005B1F6E1F7F1FCB01BA01660F771F881F6E
:10744000991F09C033E001C034E0660F771F881F21
:10745000991F3150D1F7620F711D811D911D089543
:107460000F931F93CF93DF938C01C8010E94D43CEC
:10747000EC0197FD08C00E94AA3C892BB1F7B80126
:10748000CE010E944E3DCE01DF91CF911F910F9111
:1074900008958F929F92AF92BF92EF92FF920F93B7
:1074A0001F93CF93DF938C01D62F7A01B22E0E94C7
:1074B000D43C9C0133272B32310531F02D3231057C
:1074C00061F48B2D8068B82ED15011F480E068C033
:1074D000C8010E94D43C97FDF9CFCB2DCD7F2B2D39
:1074E000207309F58033F9F4AA24AA94AD0E09F4A7
:1074F00043C0C8010E94D43C97FD3EC09C012F7D33
:1075000033272835310549F4C264D250A9F1C801A6
:107510000E94D43C97FF07C02FC0B6FE02C0C260D5
:1075200001C0C261DA2D812C912C540120ED280F6D
:10753000283080F0C4FF04C0B8010E944E3D19C03D
:107540002A3040F0C6FFF8CF2F7D3FEE320F3630A5
:1075500098F727504C2FC501B4010E94093A4B01FE
:107560005C01C260D15059F0C8010E94D43C97FF21
:10757000DDCFC1FD04C0AACF812C912C5401C7FFDF
:1075800008C0B094A09490948094811C911CA11C7C
:10759000B11C2C2FB501A401C7010E94FD3981E067
:1075A000DF91CF911F910F91FF90EF90BF90AF901F
:1075B0009F908F900895A0E2B0E0E1EEFAE30C9482
:1075C00023355C01962E7A01F9018E010F5F1F4F62
:1075D000680180E2D8011D928A95E9F7D5011396DA
:1075E0008C9080E090E0612C712C30E061E070E0E4
:1075F00083FC259183FE21918F01522E211103C01E
:1076000080E090E092C02E3511F4009751F1432FA5
:1076100050E0481759073CF42D3559F12D3219F433
:10762000772009F103C0772009F46AC0452D4695FB
:1076300046954695D601A40FB11D452D47708B0187
:1076400002C0000F111F4A95E2F7A8015C91452B7B
:107650004C93651459F0561410F45394E7CF5A9490
:10766000E5CF31E004C07724739401C0712C0196FA
:10767000BFCF772019F08E8180628E83311103C0D5
:107680008824839417C0F6019E012F5D3F4F8081AF
:10769000809581932E173F07D1F7F2CFE114F104C3
:1076A00029F0D7018C93F70131967F019A94812CB0
:1076B0009920F9F0C5010E94D43C97FD18C0FC0147
:1076C000FF2723E0F595E7952A95E1F7EC0DFD1DE1
:1076D000208130E0AC014770552702C035952795D1
:1076E0004A95E2F720FDDACFB5010E944E3D8110A8
:1076F00087CFE114F10411F0D7011C92C80115C025
:10770000422F469546954695D601A40FB11D422FAE
:1077100047708B0102C0000F111F4A95E2F7A801C4
:107720005C91452B4C93622EA2CFA096EFE00C9477
:107730003F35A0E0B0E0EFE9FBE30C9423356C01AA
:10774000EB015A01FC0117821682512CF601E380ED
:10775000FE01E3FC8591E3FE8191182FEF01882360
:1077600009F4EEC090E00E94AA3C892B21F0C601EA
:107770000E94303AEBCF153241F4FE01E3FC159143
:10778000E3FE1191EF01153281F4C6010E94D43C51
:1077900097FDD4C0412F50E09C01332724173507B3
:1077A000A9F2B6010E944E3DCBC01A3239F4E3FC77
:1077B0001591E3FE1191EF0101E001C000E0F12C11
:1077C00020ED210F2A3080F402606F2D70E080E000
:1077D00090E040E20E94093AF62EFE01E3FC15918A
:1077E000E3FE1191EF01ECCF01FF03C0F11003C0E4
:1077F000A7C0FF24FA94183619F01C3651F010C0B7
:10780000FE01E3FC1591E3FE1191EF01183641F4FE
:1078100008600460FE01E3FC1591E3FE1191EF01A5
:10782000112309F48DC0612F70E088EE90E00E9472
:10783000B33C892B09F484C000FD07C0F5018080AA
:107840009180C50102965C0102C0812C912C1E36EC
:1078500051F4F6014681578160E070E0202FC401A9
:107860000E94FD3973CF1336A9F401FD02C0FF2435
:10787000F394C6010E94D43C97FD60C0811491042A
:1078800029F0F4018083C40101964C01FA94F110AF
:10789000F0CF50C01B3559F49E01A4016F2DC601D5
:1078A0000E94DB3AEC01892B09F044C03EC0C601BE
:1078B0000E94303A97FD42C01F3661F128F4143619
:1078C00039F1193651F128C0133771F0153701F12C
:1078D00023C08114910429F0F4016082C40101964F
:1078E0004C01FA94FF2071F0C6010E94D43C3C0187
:1078F00097FD08C00E94AA3C892B59F3B601C30129
:107900000E944E3D81149104A9F0F401108212C02E
:10791000006203C0006101C00064202FA4016F2D2C
:10792000C6010E94493A811105C0F6018381807326
:1079300029F406C000FD0ACF539408CF552019F052
:10794000852D90E002C08FEF9FEFCDB7DEB7EFE05F
:107950000C943F3591110C94C53D803219F089503B
:107960008550C8F70895FC010590061621F0002007
:10797000D9F7C00108953197CF010895FC01059012
:10798000615070400110D8F7809590958E0F9F1F21
:107990000895FC016150704001900110D8F7809566
:1079A00090958E0F9F1F0895CF93DF93EC012B814D
:1079B00020FF33C026FF0AC02F7B2B838E819F813F
:1079C00001969F838E838A8190E029C022FF0FC099
:1079D000E881F9818081082E000C990B009719F439
:1079E00020622B831AC03196F983E8830EC0EA85A2
:1079F000FB85099597FF09C02B81019611F080E264
:107A000001C080E1822B8B8308C02E813F812F5FD4
:107A10003F4F3F832E83992702C08FEF9FEFDF9167
:107A2000CF9108950F931F93CF93DF93FB01238191
:107A300021FD03C08FEF9FEF2CC022FF16C04681AF
:107A40005781248135814217530744F4A081B181C5
:107A50009D012F5F3F4F318320838C932681378197
:107A60002F5F3F4F3783268314C08B01EC01FB014E
:107A70000084F185E02D0995892BE1F6D801169651
:107A80008D919C911797019617969C938E931697BC
:107A9000CE01DF91CF911F910F910895FB012381BA
:107AA00020FF12C026FD10C08F3F3FEF930761F00B
:107AB00082832F7D206423832681378121503109E1
:107AC00037832683992708958FEF9FEF0895FA0152
:107AD000AA27283051F1203181F1E8946F936E7F0D
:107AE0006E5F7F4F8F4F9F4FAF4FB1E03ED0B4E0FE
:107AF0003CD0670F781F891F9A1FA11D680F791F3F
:107B00008A1F911DA11D6A0F711D811D911DA11D4F
:107B100020D009F468943F912AE0269F112430195F
:107B2000305D3193DEF6CF010895462F4770405DFA
:107B30004193B3E00FD0C9F7F6CF462F4F70405DA9
:107B40004A3318F0495D31FD4052419302D0A9F704
:107B5000EACFB4E0A6959795879577956795BA95FE
:107B6000C9F700976105710508959B01AC010A2EC4
:107B700006945795479537952795BA95C9F7620F9B
:107B8000731F841F951FA01D0895992788270895A6
:107B9000F999FECF92BD81BDF89A992780B50895D5
:107BA000A6E1B0E044E050E00C94023EA8E1B0E071
:107BB00042E050E00C94023E262FF999FECF92BD90
:107BC00081BDF89A019700B4021639F01FBA20BDA2
:107BD0000FB6F894FA9AF99A0FBE08950396272FD4
:107BE0000E94DD3D0E94DC3D252F0E94DD3D242FBB
:107BF0000C94DD3D0196272F0E94DD3D0C94DC3D69
:107C0000DC01CB01FC01F999FECF06C0F2BDE1BD5C
:107C1000F89A319600B40D9241505040B8F708954B
:047C2000F894FFCF06
:107C24003C02FF2901AD2526040A02249A030750C9
:107C340024FA0208D824AA02043926960201010370
:107C44000303030303030303030303010303030302
:107C54000303030303030303030307F000400101C9
:107C640005012F000000000000000000000000FFDC
:107C7400FF4001F000010000005374617274005071
:107C84006175736500547572626F0045786974009C
:107C9400526F74617465005363726F6C6C00426F51
:107CA4006F744431003130353000426C616E6B00CA
:107CB40053617665496D005361766500546F7000B9
:107CC40050726576004F4B004E657874004C6173BA
:107CD400740044303A0044313A3C656D7074793E26
:107CE40020202020200044323A3C656D7074793E97
:107CF40020202020200044333A3C656D7074793E86
:107D040020202020200044343A3C656D7074793E74
:107D1400202020202000546170653A004E657700D1
:087D24003E3E3E00436667008D
:00000001FF
